:020000040000fa
:080000000002040000000000f2
:020000040000fa
:100400002fb72000807f220000018800000000003c
:10041000050007000c000700ae64020000000000a9
:100420000040da000000fe004440a90000822000e5
:100430000000e0000300320000002000a00188005e
:100440004440a80000000600e094260001002000bf
:100450001600370062004000e080480091018800eb
:100460009001ba0062004000e080480091018800dd
:100470009002ba0062004000e08048000002eb00f9
:100480006028e10005003a008301e900070033001d
:10049000038009000059eb00040037006128e100e7
:1004a000010032000082eb00050007009101880086
:1004b0001001ba000200e000e6ff3a00000005006b
:1004c000910188008002780062004000e0804800ce
:1004d0003559ba008301e900080032002559ba00f5
:1004e0008301e900050032000400e000f4ff32005f
:1004f00015d9ba008301e900f1ff3a0000000600b7
:100500001004040000000000800178000001780061
:1005100031407800005978000004e000fcff3a0008
:10052000030078000000060080007800010037001a
:100530000000e8001004e000fdff3a000100500058
:10054000000006001600fa00889fbe008a9fbe00c9
:100550008c9fbe0090bf9f00010478000206be0081
:10056000800478006e805700d3000700e805600023
:100570000030a100e10f50003e003a007a8557009c
:100580009fb89700240020008a01780008017800b5
:10059000090078004d010700000478000000e00029
:1005a00007003a006000b8006011b800f0af9f008b
:1005b00081b79f0092b79f00a3b79f002900370023
:1005c0004200dd00000045001000be00a51307003a
:1005d000f0af9f0081b79f0092b79f00a3b79f0025
:1005e0004341dd0080ff2f0000c0b9000001410041
:1005f00060ae200080044100160037004240dd005c
:10060000e1fd2f008f80400000804000d00090006e
:1006100040009000e00f5000e08f58000d003200c5
:10062000901307003902be002903be00020c070028
:100630007faa97008fb297001fb39700afb39700c0
:1006400038110700f0af9f0081b79f0092b79f005d
:10065000a3b79f000804e900e88444000800e00014
:10066000e6ff3c007a80570030024600a0824e0030
:1006700042003700e20f500046003a007a855700ea
:100680009fb89700000278008a017800080178007e
:1006900009007800ef010700000478000000e00086
:1006a00007003a006000b8006011b800f0af9f008a
:1006b00081b79f0092b79f00a3b79f002900370022
:1006c0004200dd00000045001000be006513070079
:1006d000f0af9f0081b79f0092b79f00a3b79f0024
:1006e0004341dd0080ff2f0000c0b9000001410040
:1006f00060ad200080044100160037004240dd005c
:10070000e1fd2f008f80400000804000d00090006d
:1007100040009000e00f5000e08f58000d003200c4
:10072000501307003902be002903be00c20b0700a8
:100730007faa97008fb297001fb39700afb39700bf
:10074000f8100700f0af9f0081b79f0092b79f009d
:10075000a3b79f000804e900e88444000800e00013
:10076000e6ff3c003fb19700cfb19700e0fd2f00be
:100770000f004000ac0207000c02be007fa89700eb
:100780008fb097001fb19700afb1970039030700f2
:1007900013003700e30f500004003a006000b80077
:1007a0000200200003ff270006003700e40f50007e
:1007b00009003a00f0ff2f00f1ff2f00f2ff2f0099
:1007c000f3ff2700f0af9f0081b79f0092b79f0013
:1007d000a3b79f00060037006000b8006011b800a2
:1007e000f0af9f0081b79f0092b79f00a3b79f0013
:1007f0007fa897008fb097001fb19700afb1970007
:100800000b00e0000100320003f0a2004f06be0022
:100810004f05be004f04be000080fa000000060035
:10082000881f780002047800950307000800400044
:100830004f047800000006000000fa00881f7800ce
:10084000000478003fb99700ea81570080007800e3
:100850000041200091030700800078000000e000c4
:10086000020035000040eb0000f478000100780041
:100870004f0478000080fa00000006008001780034
:1008800000017800010037000201e8001204e000d6
:10089000fdff3a00020037000201e8008100e80095
:1008a00011407800004978000004e000faff3a00a7
:1008b0000300780000000600889fbe008a9fbe00eb
:1008c0008c1f7800000678008105780010057800fc
:1008d0000a047800010037000804e8009844780012
:1008e0000900fb0026040700800078000000e000fb
:1008f000f9ff3a00d0c2b30080cf540003003a00a1
:100900000804e8008200200005003700b0c2b300f0
:1009100080cf540001003a000804e800010178008b
:1009200098407800e5c6b30085cf50000300320040
:10093000e3c4b30083cf500022003a0098409000f7
:1009400010c6b30080cf50000300320010c4b300c3
:1009500080cf500050003a00a840900085cf500052
:1009600003003200e0c4b30080cf50004a003a00d8
:100970006305440080c2b3009a4f100002003200a9
:100980000a047800090037000a047800d844780087
:100990000900fb00020407000000e000fbff3a0032
:1009a000f0c5b30080cf5400f8ff320042002000b1
:1009b00090c2b300984f100038003a000805e800d4
:1009c0003600370094c6b30084cf500003003200d5
:1009d00090c4b30080cf500034003a00184090001b
:1009e000854f500002003200834f50002a003a0029
:1009f000a840900060c6b30080cf500003003200d2
:100a000060c4b30080cf500023003a006305440067
:100a10003200b3009a40780084cf500003003200c7
:100a200090c4b30080cf50001c003a0048409000b2
:100a3000854f500002003200834f500017003a00eb
:100a4000d840900084cf50000300320090c4b3001f
:100a500080cf500011003a00e840900040c7b3003a
:100a600080cf50000300320040c5b30080cf50005b
:100a70000a003a00f840900090c7b30080cf5000c1
:100a80000300320090c5b30080cf500003003a004d
:100a900068054400010037000001eb000b00e00096
:100aa000040032008a0d7800020037000200a00026
:100ab000080578000a0e7800020078004f067800da
:100ac0004f05be004f04be0000000600e48747004b
:100ad000889fbe008a9fbe008c9fbe008e1f78003c
:100ae00080bf9f0081047800020778000306780029
:100af0006922b900040578008006eb000200370087
:100b00008904e8001d00200000c3b300994f1000c5
:100b1000fbff3200000eeb003c1678000c0478005e
:100b20008005eb00280037008a8f550016003d0035
:100b300092002000110009008205d8000100780011
:100b40000000e00003003a0064044400000ceb00e5
:100b500038147800a2002000030020001800be0016
:100b6000c0140700194178000201fb00cf91de009c
:100b700000004100818049000003b1000180b10004
:100b8000008cbe000d003700100020000100200086
:100b90001c0e40005c9648008a8f550008003a0001
:100ba00040c3b300994f100005003400100020002e
:100bb00001002000180c4000589448008b05e80004
:100bc0008904e8001d002000194178000200fb00a4
:100bd0000003b100e90f5000d3ff36008b0f550022
:100be00001003d008a057800e0c2b300804f51004b
:100bf00001003a008904e8000b00e0000700320021
:100c0000290037000080eb008080eb001c0e4000c4
:100c10005c9648008904e8001d00200000c3b30072
:100c2000994f1000f7ff32008005eb001e003700df
:100c30008a8f55001a003d00920020001100090023
:100c40008205d800010078000000e00003003a00af
:100c500064044400000ceb0038147800a20020006b
:100c6000030020001800be007e1407001941780020
:100c70000201fb00cf91de000000410081804900ad
:100c80000003b1000180b100008cbe008b05e800bc
:100c90000080eb008080eb001c0e40005c9648005a
:100ca0008904e8001d0020001900fb000003b100ca
:100cb000e90f5000deff360092002000110009000d
:100cc0008205d800010078000000e0001700320023
:100cd000690510001802be00e00f5200e08f5a00b4
:100ce000070032004250dd00a1af200001004000ab
:100cf0001001be000400be005a140700008cbe00a4
:100d00008a8545006150b9001c1e10001c96180011
:100d100006003700e9855500900020000100200002
:100d20001c0e40005c96480064045400e88f550097
:100d3000040034001800be00e00f5000e08f58009f
:100d4000f4ff32000d00e0003300320099407800db
:100d500050c6b30080cf50000300320050c4b3002f
:100d600080cf50002c003a008900e8001144780040
:100d7000b2c2b300824f540006003200d0c2b300aa
:100d8000804f540003003200810478000244780050
:100d9000010037008984e8008006eb006022b8007b
:100da00011003700f00f2e00515f2000800f52001d
:100db000818f5a000a003c00a2002000030020009e
:100dc0000400be00271407000a01fb00cf91de00db
:100dd00000024100818249000403b1000580b10096
:100de0008904e8001d002000194578000a00fb0076
:100df0000003b100e90f5000eaff3600d0c2b30093
:100e0000804f540002003a0060021200e0821a0093
:100e10001c0e42005c964a000e00e0000400320006
:100e20000d00e00001003a008fbc9700090f780028
:100e300092002000110009008205d8004f077800b9
:100e40004f06be004f05be004f04be004f00b1006c
:100e500000000600e8874700889fbe008a9fbe000a
:100e60008c9fbe008e1f780080bf9f008104780099
:100e700002077800030578006722b90004067800ad
:100e80008006eb00020037008904e8001d00200006
:100e900000c3b300994f1000fbff3200000deb00c0
:100ea0003a1578000a0478008005eb002c00370022
:100eb0008c8f550019003d0072002000811f7800c2
:100ec000110009008205d80001007800cf007800e9
:100ed0000000e00003003a0064044400000ceb0052
:100ee000381478001801be004418dd00cc11de0073
:100ef000830170004411dd0040aa200000805000f2
:100f0000e1a8200060c078000000fb00cf80de0078
:100f1000001c4100019449000e003700120020001f
:100f2000030020001a0d41005a9549008c8f55008e
:100f300009003a0040aa200000805000e1a82000eb
:100f400060c07800e74f500003003400180c4100e7
:100f5000589449008b05e8008904e8001d00200032
:100f60009900fb006201200040aa20009a020700bd
:100f7000800078000000e000cdff3a008b0f5600a3
:100f800001003d008c057800e0c2b300994f1000cd
:100f900001003a008904e8000b00e000070032007d
:100fa0002c0037000080eb008080eb001a0d400021
:100fb0005a9548008904e8001d00200000c3b300d2
:100fc000994f1000f7ff32008005eb002100370039
:100fd0008c8f55001d003d0072002000811f78009d
:100fe000110009008205d80001007800cf007800c8
:100ff0000000e00003003a0064044400000ceb0031
:10100000381478001801be004418dd00cc11de0051
:10101000830170004411dd0040aa200000805000d0
:10102000e1a8200060c078000000fb00cf80de0057
:10103000001c4100019449008b05e8000081eb0091
:101040008081eb001a0d41005a9549008904e8009f
:101050001d0020009900fb006201200040aa200032
:101060005d020700800078000000e000d8ff3a0031
:1010700072002000110009008205d80001007800ec
:101080000000e00014003200670010004202dd00a2
:101090001801be000402e900030033000201410010
:1010a00083814900fbff3700028cbe00808545002c
:1010b000cf80de001a1d10001a95180006003700b8
:1010c000e785550070002000010020001a0d400047
:1010d0005a95480064045400e68f5500040034001b
:1010e0001800be00e00f5000e08f5800f4ff3200ff
:1010f0001a00be004209dd00ce01de00830171004e
:101100004201dd00e2b79f00f3b79f00028dbe00f1
:101110000d00e000350032009940780000c7b300b0
:1011200080cf50000300320000c5b30080cf5000d4
:101130002e003a008900e80011447800b2c2b300e2
:10114000824f540006003200d0c2b300804f5400da
:101150000300320081047800024478000100370067
:101160008984e8008006eb006022b8001100370097
:10117000f00f2e00515f2000800f5200818f5a0027
:101180000a003c00a2002000030020000400be0072
:10119000341307000c01fb00cf91de000002410078
:1011a000818249000403b1000580b1008904e80090
:1011b0001d002000194678000c00fb000003b10060
:1011c000e90f5000eaff3600d0c2b300804f540050
:1011d00002003a0060021200e0821a006fb097002d
:1011e000ffb09700041d4000059548000e00e00088
:1011f000040032000d00e00001003a008fbc9700af
:10120000090f780072002000110009008205d80043
:101210004f0778004f06be004f05be004f04be00ca
:101220008f00b10000000600889fbe008a1f780072
:101230008c9fbe00000478000206be00e604400059
:10124000190178000200d0004505de008a00780010
:10125000f07f2000800f55000c003a006f00610005
:1012600065003a00280090000000e00062003a00ab
:10127000180090000000e0005f003a00100020001d
:101280001800e0005d0032005b0037000a00e0005b
:1012900007003a0008007800da01070080007800b3
:1012a0000000e000020034000a007800530037001c
:1012b0006108b9000c0140008d814800e07f2000ea
:1012c000800f5100e08f59000d0034001900e0003c
:1012d00004003d006000b8000200200003ff2f0062
:1012e000030037006000b8000200200003ff270061
:1012f000009cbe000294be00100020003f0037009a
:10130000e00f5100e08f590005003400f000280084
:1013100019006000c410dd00810c7000340037003b
:101320001900780001002800010360006f006000d0
:101330000040a000800c780061015100e08159005c
:10134000c0fc2f00f1ff2f00800f5100818f59004a
:101350000d003d00860c78000000eb002004980092
:1013600010049800000c7800240037008880e80002
:10137000110c780064004400900878001908780087
:10138000800ceb0070014100f00f4100f7ff3400ca
:101390008202ea00150032008881e80070821200a3
:1013a000980078008508de00130078000400dd0056
:1013b000008c700064014400930078008508de0012
:1013c000120078000400dd0080897000920078002f
:1013d0008508de00190078000400dd000089700037
:1013e000190078000500de00800c7800990c73006d
:1013f0000080eb0001003700200020004f06be00f7
:101400004f0578004f04be00000006000200fa00fd
:10141000889fbe008a9fbe008c1f7800000678005f
:101420000404be000605be00800078006c805700f2
:10143000c00107003c02be002c03be000800be0035
:101440000a01be007c080700009ebe000296be0096
:101450002fb99700cf91de000c00780072ff0700d3
:101460004f0678004f05be004f04be000080fa0012
:10147000000006000800fa00889fbe008a9fbe0098
:1014800080bf9f0091bf9f00a2bf9f00b3bf9f007e
:101490000404be00e00f5200e08f5a0070003200da
:1014a0006022b8006033b800320907000000e00095
:1014b0006b003200e00f5400e08f5c0033003d0011
:1014c00060041400e0841c006000b80002002000ea
:1014d00003ff23008005eb00ea9f2000090037008e
:1014e0000808a300030032003a02be002a03be002f
:1014f000510807008904d1000884d3008b05e80057
:1015000068054500e00f5400e08f5c0002003200e7
:10151000e78f5500f2ff36000002be000203be0056
:101520006000b8000200200003ff2300b708070096
:101530000002be000203be0070805700b3ff070028
:10154000000578000000e0003e003d00e00f540080
:10155000e08f5c004200320034f42600c54a2600c9
:101560008662200087ac200070805700a7ff07002c
:10157000000578000000e00032003d0061045400e6
:10158000e0845c0032003200f3ff3700e00f5400cb
:10159000e08f5c002b0034008005eb006000b80099
:1015a0000200200003ff2300ea9f20000808a30098
:1015b000030032003a02be002a03be001e080700e4
:1015c0008984d1000884d3008b05e80068054500b4
:1015d000e00f5400e08f5c0002003400e78f5500fc
:1015e000f2ff36000002be000203be00708057000a
:1015f00086ff0700000578000000e00011003d00b4
:10160000e00f5400e08f5c0015003400c4f32b00a1
:1016100035f72700d6fd240057512700708057006a
:101620007aff0700000578000000e00005003d009b
:1016300061045400e0845c004240a90004003400ce
:10164000f2ff3700000120000a00e0000300320032
:10165000e10f550002003a00800020006101070000
:101660000fb897009fb897002fb99700bfb99700a0
:101670004f05be004f04be000080fa0000000600c7
:101680008001780002003700b15978000201e900ba
:101690000200e000fcff3a00000006006200fa00d1
:1016a000889fbe008a9fbe000004be00020578002d
:1016b0008300780060f92f000f00400054010700fc
:1016c00088979f0099979f000000eb00a09f9f00c4
:1016d0009a4578000b80fb000000ea00cf04de0092
:1016e00050c2b30080cf55000200320009047800d8
:1016f000010037000904e9000800e0000b00340095
:101700001f909700080178008a0078008f91970059
:101710000300010090979f000000e000930032005a
:101720002f98970000004400a09f9f0009054500e6
:1017300050c2b30080cf5500040032000b04e0001b
:10174000e3ff3a002f989700890037000000eb0074
:10175000809f9f00f0979f00e0979f00d0979f0089
:10176000c0979f00b0979f00c09f9f00090037005f
:10177000a0b220000080500000004000e1b1200035
:10178000e08078004f98970001007000c09f9f0094
:101790000a05e8001a4478008800fb00a0b2200087
:1017a00020010700800078000000e000f0ff3a0010
:1017b000a0c2b300804f54000e003a00bf889700cb
:1017c0000180e900b08f9f0010007800b09f9f005b
:1017d0000000e00005003d000000ea00b09f9f000f
:1017e0004f9897000020a000c09f9f000a05e800c6
:1017f00010003700b19f9f0009003700bf98970085
:10180000f0ff2700808f5000040032006a08b90002
:101810000000410003004000b09f9f000a05e8005f
:101820001a01fb0003fd2f0003004100e90f5000e7
:10183000f2ff3600e0c2b3009a4f100004003200fd
:101840000080eb00909f9f008a0478001c00370006
:101850008a04e800a0c2b300994f100007003a00c4
:10186000bf8897000180e900b08f9f0010007800ca
:10187000909f9f008a84e800110037000000eb0071
:10188000909f9f00090037009f989700f0ff270066
:10189000808f5000040032006a08b9000000410047
:1018a00003004000909f9f008904e8001901fb009d
:1018b00003fd2f0003004100e90f5000f2ff360046
:1018c000194478008800fb0080b62000d50007008e
:1018d0000000e00002003a000044780001003700f8
:1018e0008904e800a87f9f0080c6b300804f5400a1
:1018f00004003a00994f14000a003a006640500074
:1019000006003700c0c6b300804f540005003a00ff
:10191000994f140003003a0065404000a07f9f00eb
:101920008904e8000905e800cbfb2f008f854500fe
:101930001901fb0060f92f000f0040000084e8004f
:101940008b0178008000780008007800be00070056
:101950000000e00005003a008b00780008007800e5
:101960002d0207000000e00059ff3d000080eb0061
:101970004f05be004f04be000080fa0000000600c4
:101980006900e100040035006d00e100030034004f
:101990000002b10001003200000005001000050047
:1019a0000003b1000b0035009000b10008003400c6
:1019b0008000b100070035009001b1000400340040
:1019c0007000b100030035009001b10001003c003f
:1019d00010000500000005000600370090cf100041
:1019e00002003a0000017800040037000000e8001f
:1019f0000201e9000200e000f8ff3a00020078006e
:101a00000000060000027800e602400015007800a1
:101a100001002800810360006f006000800a7800e8
:101a200012003a00240090000000e0000f003a008d
:101a3000140090000000e0000c003a0016002000a6
:101a40001400e0003800320008003700e4004200d3
:101a5000910a78000480e800900878001408780063
:101a6000000aeb007003530001003700160020004d
:101a70001500e000f5ff320013003700640142005a
:101a800080004000120078004f00de00808a700065
:101a90008481e80092007800818040001300780083
:101aa0004f00de00008970009300780081804000c4
:101ab000140078004f00de00808970001400780068
:101ac000000a40000603e90015007800ef0f5000ff
:101ad000eaff3600100037000481e8009400d100ce
:101ae000120078004f00dd00008a7000e400420020
:101af0009201d100110078004f00dd0000897100d3
:101b00001101d100150078004f00dd008008710040
:101b1000950ad1000603e80015007800ff0f500079
:101b2000edff3e00ef0a6000958a73000600780022
:101b300000000600889fbe00800478006684400094
:101b400000ff2700180060004401de00f07f200045
:101b5000800f51000e003a00800ceb001804780052
:101b60006f0064001c003a00210090000000e000bb
:101b700019003a00110090000000e00016003a0041
:101b8000100020001100e0001400320012003700a5
:101b90000200e00005003c000100780099ff07000a
:101ba000000178000000e00008003c00f000280080
:101bb0001800600001fe2300010c700020c02f00ff
:101bc000800c41000080eb0004003700800ceb002b
:101bd0000000eb0001003700200020004f04be0091
:101be00000000600800078006500600003003200fd
:101bf00010022000805988000000060078806000f4
:101c000002003200200220008059880000000600f7
:101c10000200fa00f1bf9f00010878000080fa007e
:101c200000000600040037000204e00001003a0052
:101c3000000005000000e80010417800814f5100cd
:101c4000f9ff3a0000000600889fbe008a1f780056
:101c500000047800010278008244780003057800cf
:101c600070c6b300804f510021003c0000c0e90065
:101c7000804f5100df003d0072405000804f510006
:101c8000420132000d003c006c405000804f51007a
:101c900055013c0000c0e900804f5100d5003d00d7
:101ca00050c2b300804f51004c0132007c404000d4
:101cb000804f51004c013a00ce00370010c6b300ef
:101cc000804f5100cb00320004003c0069405000be
:101cd000804f510044013a007200370030c6b30013
:101ce000804f5100180032000040e8000900370022
:101cf00000c7b300804f51001501320008003c00be
:101d000000c0e900804f5100db00320065003c005c
:101d10006540500080cf540033013a000f00370077
:101d200050c7b300804f51005e0032006340400056
:101d3000804f51005b00320065405000804f5100e1
:101d400029013a00110137009180e900010a780069
:101d5000780090009171780029013700a860900008
:101d6000c0c6b30080cf50000a003a00940078004b
:101d700064805000000a78001000be004f89de0029
:101d8000cf91de000002be000203780082037800db
:101d90001300370010c7b30080cf5000030032009b
:101da000a0c6b30080cf500006003a00940078002f
:101db00068805000000a78003002be002003be0098
:101dc000070037001480e900000a7800100078004e
:101dd00000027800cfa2de000503780086037800b9
:101de000049cbe000694be00a860900080c6b300ac
:101df00080cf50000e00320020c6b30080cf5000cc
:101e000005003a000400fb00cf80de0001017800ed
:101e1000820178000a00370040c7b30080cf50002d
:101e2000030032006640400080cf500006003a00b8
:101e300004007800cf80de00010178008201780084
:101e4000009cbe000294be003800be002801be0007
:101e5000e00f5000e08f5800e00f5900e08f59006c
:101e600003003d0078009000d1c2b3000a003700a3
:101e7000081090000018a3000300320078009000c2
:101e8000b1c2b300040037000008a30054003200c0
:101e90007800900001c2b300017578000000e800ee
:101ea0004e003700a8609000c0c6b30080cf50003d
:101eb00007003a009400780064805000000a78001f
:101ec0001002be000003eb00860378001300370009
:101ed00010c7b30080cf500003003200a0c6b3008b
:101ee00080cf500006003a009400780068805000cf
:101ef000000a78003002be002003be000700370051
:101f00001480e900000a78001000780000027800d0
:101f1000050020000600200007002000049cbe00f1
:101f20000694be00a860900080c6b30080cf500029
:101f30000e00320020c6b30080cf500005003a00ea
:101f40000480fb00010020000200200003002000ac
:101f50000a00370040c7b30080cf500003003200b2
:101f60006640400080cf500006003a000400780030
:101f7000010020000200200003002000009cbe00a1
:101f80000294be00081090000038a3001400320034
:101f90003800be002801be00e00f5000e08f58005e
:101fa000e00f5900e08f59000d00320080c7b300e8
:101fb00080cf54000300320080c5b30080cf5400ae
:101fc00007003a007800900001c3b3000175780063
:101fd0008000e80009f578000080e80070049800af
:101fe0007800900000004500600498008940780067
:101ff000630037001400780068015000020a78007e
:102000003200be001201be00009cbe000294be0061
:10201000380090000000e00003003d0078009000d0
:10202000d1c2b3000a003700081090000018a300c6
:102030000300320078009000b1c2b3000400370002
:102040000008a300050032007800900001c2b30030
:10205000017578000000e800700498007800900096
:10206000000045006004980089407800080078006e
:102070003301070064003700a8609000c0c6b300b9
:1020800080cf5000250032000a003c006440500020
:1020900080cf50002800320000c0e80080cf500000
:1020a000140032006840500080cf500022003a00f7
:1020b0000a00370040c7b30080cf50001e00320036
:1020c0006640400080cf50001b0032006940500045
:1020d00080cf500018003a00060037001480e90055
:1020e000000a780010007800485c900008487800ea
:1020f000450037001480e900000a780010027800db
:1021000068089000cf80de0001017800820178002d
:10211000009abe000292be003b0037001480e90026
:10212000000a78001001780068089000cf80de0077
:102130000089be00340037001480e900000a7800ee
:1021400010007800680c9000080878002e00370016
:102150001180e9008008780010007800cf80de0050
:102160000101780082017800009cbe000294be004c
:1021700078009000000045006004980081c7b3001b
:1021800008007800160307001f0037001480e900dc
:10219000000a780010007800600498005809900048
:1021a0000200e00002003d00dff8070009003700f0
:1021b0008000eb0008fe0700800078000000e000cf
:1021c00003003200680090000080500001003700da
:1021d00058089000100c98000b0037007800900011
:1021e00002757800060037007800900080004500f6
:1021f0000904e00001003a0059c2b30089487800a0
:102200000000e800700498000000eb004f05780023
:102210004f04be00000006000400fa00889fbe00c4
:102220008a9fbe008c1f78000004780001067800a9
:1022300070089000f800900001005000880890009d
:10224000010050009808900001005000a80890007c
:1022500001005000b808900001005000c80890002c
:10226000810550000002220090bf9f000003230060
:10227000a0bf9f00081090000028a30018003a009b
:102280000b00e000160034008b047800090578008c
:10229000e28f5400020036002a00200002003700be
:1022a0000900e0000b00340058009000c8019000c5
:1022b0000a017800ee8057000300010050049800e6
:1022c0000000e00096003200680890000000450021
:1022d000600c98008a8454004240a900ebff3c0047
:1022e000780190000200e0000b00340058009000dc
:1022f000c80190008c007800030001005004980091
:102300000000e0008600320068089000f8009000ad
:1023100001004000600c9800880c90000900e0006b
:102320001500340009057800e28f540002003600e1
:102330002a002000020037000900e0000b003400f2
:1023400058009000c80190000a017800ec80570006
:1023500003000100500498000000e000700032000b
:102360006808900000004500600c98008a845400c2
:102370004240a900ebff3c00180990000200e00079
:102380000b003400e800900058009000c801900055
:1023900003000100500498000000e00060003200db
:1023a000680890009808900001004000600c9800b8
:1023b000a80c90000900e000150034000905780021
:1023c000e28f5400020036002a002000020037008d
:1023d0000900e0000b00340058009000c801900094
:1023e0000a017800ec8057000300010050049800b7
:1023f0000000e0004a00320068089000000045003c
:10240000600c98008a8454004240a900ebff3c0015
:10241000380990000200e0000d003400e800900050
:10242000180890008080400058009000c80190007b
:1024300003000100500498000000e0003800320062
:1024400068089000b808900001004000600c9800f7
:10245000c80c90000900e000150034000905780060
:10246000e28f5400020036002a00200002003700ec
:102470000900e0000b00340058009000c8019000f3
:102480000a017800ec805700030001005004980016
:102490000000e000220032006808900000004500c3
:1024a000600c98008a8454004240a900ebff3c0075
:1024b000081090000028a3001b0032000b00e00071
:1024c000190034008b04780009057800e28f54006d
:1024d000020036002a002000020037000900e00058
:1024e0000b00340058009000c80190000a017800e9
:1024f000ee80570003000100500498000000e00047
:10250000070032006808900000004500600c980049
:102510008a8454004240a90003003400eaff3700d7
:102520000080eb00010037000000eb004f06780050
:102530004f05be004f04be000080fa0000000600f8
:102540000f05b000889fbe008a9fbe008c9fbe0012
:102550008e1f7800f0b79f0081f79f005001be00ea
:102560004000be00b0979f00c1979f00d2979f0088
:10257000e3979f0010c6b3000ff19700804f510002
:102580001600320010c4b300804f51001300320017
:10259000ffb19700530890000000e00003003d00e9
:1025a00060002000d00998000c0037000000e00017
:1025b0000a003a0070c6b3000ff29700804f520035
:1025c0000300320070c4b300804f520003003a0091
:1025d00010002000ffb29700d00a9800ffb09700cb
:1025e00040fa2f000f00400052fd070080017800e4
:1025f000e20f500015003a0030002000ffb09700b5
:102600009008980010c6b3000ff19700804f51005a
:102610000a00320064404000804f51000700320041
:102620000040e800804f51000400320061b32000f8
:102630000040e800804f510001003a00a1b32000a3
:10264000ffb1970063009000160037000000e00023
:1026500018003400300020007fb29700100a980064
:1026600010c6b3008ff2970080cf52000a003200ec
:102670006440400080cf5200070032000040e80074
:1026800080cf520004003200e1b320000040e80097
:1026900080cf520001003a0021b420007fb19700a2
:1026a0006200900031587800315878001148780065
:1026b000c501370014c6b3008ff2970084cf5200d3
:1026c0000300320010c4b30080cf520013003a0060
:1026d0007fb09700600190008200780000c3b300d3
:1026e00080587800ffb29700e102980080c7b300dd
:1026f0008ff2970084cf52000100320080c5b300f2
:10270000804878000280e800ffb09700e000980061
:10271000710090000080e800f00098000300e000e5
:1027200005003a00a3979f0064fb2f000f014200b1
:10273000030778009f01370065b42000e5b79f00cc
:1027400010c6b3008ff0970080cf50000500320014
:1027500010c4b30080cf50009f003a0072b5200033
:10276000e2b79f00ffb19700530890001e022000bf
:102770000000e000010035000007e8000e02e8005c
:10278000d4b79f006022b8006033b8003f90970034
:10279000cf9097005f919700ef9197007504070025
:1027a000ffb097003102be002103be000000e00030
:1027b00004003d000400be000601be0003f0a200bc
:1027c000020037000400be000601be00b0979f0063
:1027d000c1979f00d2979f00e3979f002f9197008a
:1027e00064015100a2979f0043fa2f008f8141009e
:1027f000728041000048eb0073824100c4b79f0023
:1028000030003700c20120000300200065fa2f00cd
:102810000f80420084fa07003f949700cf949700fe
:102820005f959700ef9597000800be000a01be0073
:102830000f0b07000006be005fb197006701510053
:10284000d2b79f004240a9000a003400050b0700e0
:102850000002be000203be000800be000a01be0066
:10286000a9080700b0979f00c1979f00d2979f00cb
:10287000e3979f00cfb1970067804100710020006f
:10288000050037006f6066004c6add004466de00bc
:102890000c067200c4eede00e00f5600e08f5e0012
:1028a000040034008100e900f6ff3b00010037001e
:1028b0000060eb008100e900fdff3b006700400085
:1028c000c0b79f00dfb297000500e00009003400a8
:1028d0006022b8006033b8003f909700cf90970017
:1028e0005f919700ef919700890807000000e000d2
:1028f000c4ff3c0060fb2f008f0040004fb19700e9
:10290000010051000000e9008e0f500001003d0061
:10291000000778000e00e00003003d0073fb2f006d
:102920000f81410025003700800f570005003d0052
:102930000e80400010409000f4c0b300e74f5000fc
:1029400001003c000042eb000e007800010037005f
:102950000e07e9000000e90075fb2f000f8142001f
:10296000800141009340780084cf5000f8ff32008e
:10297000ef4f520001003a008149e8000000e000fa
:1029800006003d000e07e8002f909700640040000d
:10299000a0979f0061fb2f000f8140008e017800ff
:1029a00004003700830041001100fb006fb2970064
:1029b000e44878008301e900faff3b00ffb297008a
:1029c000550890000000e000fa003d000e00e9000c
:1029d000d00a9800f70037003f949700cf949700f3
:1029e0005f959700ef9597006022b8006033b800bc
:1029f0000800be000a01be00de0307000000e00080
:102a000005003d000bf0a200b8979f00c9979f00fa
:102a1000da979f00eb979f002f909700725927003d
:102a20000280b900026a280013002000130d07007d
:102a3000e4005000a1979f0019003b00e3801000c4
:102a4000c0ff2f00008460000800ea00a0979f00ec
:102a500069a420000f0037000808a3000b00320013
:102a60003902be002903be003f909700cf90970027
:102a70005f919700ef919700ef020700b0979f00da
:102a8000c1979f00d2979f00e3979f000884d100d1
:102a9000e88444000800e000efff3c001f0037001e
:102aa0000100e0001d003400c0ff2f000080600026
:102ab000a0979f00000478006000b800020020008a
:102ac00003ff230069a42000070037000808a300c3
:102ad000030032003902be002903be00d6020700ff
:102ae0000884d100e88444000800e000f7ff3c00bf
:102af0000002be000203be003f909700cf909700f7
:102b00005f919700ef91970040030700b0979f00f7
:102b1000c1979f00d2979f00e3979f00ffb0970057
:102b20005109900060c6b3008ff1970080cf51002b
:102b3000040032006100200060c4b30080cf510067
:102b400002003a002f929700ea004200010741007c
:102b5000f30f5700010034003e01200000c3b30012
:102b6000e0779f0075fb2f008f824200b5b79f0072
:102b7000390037000800be000a01be003c0a070009
:102b80000006be00680757004240a9000e0034004e
:102b9000340a07000002be000203be000800be00a7
:102ba0000a01be00d80707006022b80046782d0051
:102bb00077192400a0020700b0979f00c1979f00db
:102bc000d2979f00e3979f003fb0970068054000b1
:102bd0008b0020001400370041fa2f008f80400046
:102be000ea84400001047800a803b000a40020009b
:102bf000050020000c01be00080078002f0107002e
:102c00001801be00828cbe001fb29700afb29700c1
:102c1000949f9f00a59f9f002f70970005c3b3004e
:102c2000056540001906be00e00f5600e08f5e000b
:102c3000050034008b05e900e7ff3b000200370088
:102c400000c3b300006578008b05e900fcff3b0082
:102c500068054500bab79f000e00e0000b00340085
:102c60003f949700cf9497005f959700ef9597005a
:102c70006022b8006033b8000800be000a01be0040
:102c8000a30707000000e000baff3c0041fa2f0054
:102c90008f804000728040003fb1970000005100db
:102ca0000002e900af919700e7814100a3979f00e0
:102cb00073814000050037000402e900af929700dd
:102cc0008502e900a5979f000201e80000c3b30058
:102cd000924f1000f8ff32007fb09700d0099000ab
:102ce00060c6b3008ff0970080cf50000300320021
:102cf00060c4b30080cf500003003a00af92970049
:102d00008500e8000a00370050c6b3008ff0970036
:102d100080cf5000050032008000eb0050c4b300ab
:102d20008ff2970080cf520001003a00110020007e
:102d3000018741008e0f520001003d00040778001a
:102d40000e00e0001b003500840f570005003d0019
:102d5000e2407f0095c3b30040c3b30080cf500072
:102d600001003c0005c3b3008e007800010037006d
:102d70000e07e9008100e90001024100944178005a
:102d800085cf5100faff320090c3b30080cf5200cc
:102d900001003a00034ae8000100e00005003d00a0
:102da0000201e9000e07e8002f9097000000e800fc
:102db000a0979f002f9297008e0178008ff09700c8
:102dc0007fb09700da0007004f0778004f06be007b
:102dd0004f05be004f04be000f05b1000000060005
:102de000ef02b000889fbe008a9fbe008c9fbe008d
:102df0008e1f78008006780000012000b0b79f0089
:102e0000d2ac2000c2b79f0080c5b30080cf500075
:102e10000e00320083002000b3b79f00c4ab200037
:102e2000c4b79f007740400080cf500007003200b9
:102e300000012000b0b79f0080c7b30080cf5000d2
:102e400002003200a2002000b2b79f003d04be0085
:102e50002d05be0040c6b30080cf500003003200f5
:102e60006540400080cf50000b003a00e00f540056
:102e7000e08f5c00e00f5d00e08f5d0006003d002c
:102e80006000b8006011b800080450008984580040
:102e90000a0559008b855900e00f5400e08f5c0053
:102ea000e00f5d00e08f5d0004003a005d089000d7
:102eb0008e0120000000e0000c003200bfb197003e
:102ec00003027800cfa2de000503780086037800b5
:102ed0000800be000a01be00800c07004fb2970038
:102ee00064407800d0df9f007e0120003fb0970053
:102ef00000027800cfa2de00050378008603780088
:102f00000800be000a01be006d0c07002300370058
:102f1000bfb0970001047800cfc4de000905780037
:102f20008a0578000802be000a03be007fa8970049
:102f30008fb097001fb19700afb197006b0c0700df
:102f4000d0b79f00e1b79f00f2b79f0083bf9f00fb
:102f50000e07e90062fc2f000f0141000e06410040
:102f60000802be000a03be005fb09700efb09700f2
:102f70007fb197008fb99700d80c07007faa970000
:102f800000005200cfb09700614e78005fb097000c
:102f9000efb097007fb197008fb99700809ebe0079
:102fa0008296be003d00be002d01be00f0af9f0026
:102fb00081b79f0092b79f00a3b79f00e00f50001a
:102fc000e08f5800e00f5900e08f590002003400f4
:102fd0000e00e000ceff3c00bfb09700e88f50002d
:102fe00010003a000d1090000038a3000d003200d0
:102ff000f70f570006003e0062fc2f000f01410052
:103000008e00410000c3b300914f10000500320054
:103010000e07e90000c3b30063fc2f008f8141005d
:1030200080717f0078011700920e98006d0090006b
:1030300063fc2f008f8141008e80410090f90700d2
:103040001d0990005d089000800f510006003d00b2
:1030500002005000800e98000d1090000040a1006a
:10306000801698000f0037000000e0000d003d00c2
:103070000d10900074006000f00f500009003a003d
:103080007d089000fd009000010050008d08900028
:1030900001005000020050004240a900010034002d
:1030a000800e98004f0778004f06be004f05be0007
:1030b0004f04be00ef02b100000006000400fa0059
:1030c000889fbe008a9fbe008c1f78000006780093
:1030d00092bf9f00a3bf9f000404be000401be0076
:1030e0001fb89700afb89700640b07000005be003b
:1030f0000001be000800be005a0b07001fb9970070
:10310000afb9970000005100818059002006980057
:10311000310698000a8ebe000c0078004f06780039
:103120004f05be004f04be000080fa0000000600fc
:10313000f4874700889fbe008a9fbe008c9fbe0018
:103140008e1f780080047800014578000206780020
:1031500003047800040778000300e00002003c004c
:10316000180020000cb7200060c6b300804f550047
:103170000e00320060c4b300804f55000b003200d7
:1031800070c6b300804f55000300320070c4b30016
:10319000804f55009c003a00e40f47008000350046
:1031a00059089000800f57007d003d008e05e80013
:1031b00060c6b300804f55001000320060c4b300f9
:1031c000804f55000d003200091090000038a30018
:1031d00004003a0059089000800f540001003d009f
:1031e000d80c9800590890000b005000d00c9800a3
:1031f00002003b000000eb00d00c98000b00e00048
:1032000027003c00190990006900900001c3b30039
:10321000017079008201e800930c98005908900031
:103220000000e00003003c00091090000038a300fb
:103230000500320069009000e1c2b30001f079009e
:103240000280e800900c9800d90890000b00ea007a
:10325000808f500001003d008105ea000b00ea006c
:10326000a00c980001804500d00c9800880f5000f9
:1032700001003d0000047800b80c9800690090003f
:103280009908900001004000080178008c00780047
:10329000fbf8070059089000080050001a0037009a
:1032a00099089000690090008b0f540018003d00b1
:1032b00001004000080178008c007800f0f8070059
:1032c0001908900000014400920c980008805500f5
:1032d000a00c9800590890000000e00003003c009a
:1032e000091090000038a30006003200e9009000a9
:1032f000e0c2b30080707900390890000000e80057
:10330000b00c980059089000c00c9800a700370036
:10331000010040000b0178008c007800d8f807000d
:103320001908900000814500920c98000b0454008d
:10333000590890000000e00003003c0009109000d4
:103340000038a3000500320069009000e1c2b3001c
:10335000017079000200e800900c98005908900074
:10336000880f500001003d000004780069009000c3
:1033700099089000010040008b0046000801780089
:10338000bff807001908900000004400900c980056
:103390005908900008005000a00c980083003700e6
:1033a00070c6b300804f55000300320070c4b300f4
:1033b000804f550014003a0059089000800f5400c7
:1033c00004003d00091090000038a30001003a00fd
:1033d000d80c9800590890000000e900d00c980023
:1033e00002003b000000eb00d00c980070c6b30058
:1033f000804f550002003a005ac6b3000b00370058
:103400005ac4b3000900370010c6b300804f5500fe
:1034100002003a000ac7b3000400370010c4b3002a
:10342000804f550001003a000ac5b3001909900009
:10343000690090003c7079008201e800930c9800cc
:103440000c027800590890000000e00003003c00e6
:10345000091090000038a30017003200e900900026
:10346000e0c2b30080f079008280e800910c9800ff
:10347000590890000000e0000f0034000804e90043
:10348000880f500001003d000004780069009000a2
:1034900000804000080178008400780078f8070078
:1034a0001908900000004400900c98005908900002
:1034b00008005000a00c9800690090009908900046
:1034c000010040008086e8000a58780080007800fb
:1034d0000e00e00004003500b0c2b3008048780060
:1034e0008d05780004003700d0c2b3008048780012
:1034f0008d0578000e07ea000006eb000d0037008e
:1035000072845700a20020008e0078000800780026
:103510003e00070000fe2f000f0040001801be0013
:103520000298be00afe1970003707e000fb79700ce
:103530000c06e8000e00e000f1ff3c00e10f560031
:103540000e003c0050c6b300804f5500030032000f
:1035500050c4b300804f550003003a0000c3b300cd
:10356000805e78008d0578000c00e00008003a00cd
:1035700000c3b300805d7800070037000c06e90047
:103580007c8057000c00400001c3b30090dd400078
:103590000c00e000f9ff3c006900900099089000e1
:1035a0000100400000805500b00c98000910900008
:1035b00074006000f00f50000e003a007900900097
:1035c0009908900001004000a90890000100400007
:1035d000b908900001004000c90890008100400037
:1035e00079089000808f500002003d0001005000db
:1035f000800c98004f0778004f06be004f05be00b4
:103600004f04be004f01b100000006000202780026
:10361000809fbe00110009008200d80000017800e0
:103620004f00be0002a2b900848050001100980033
:1036300002087800000006002800fa00889fbe00fb
:103640008a9fbe008c9fbe0003866b004a0607005f
:103650000028a30064003a000128a30067003a0094
:103660000008a30062003a000108a30065003a00c8
:103670001e009000be08900081064000ed3fb100a2
:10368000f4805700ee019000111ab8008e099000e6
:10369000311bb8009e099000311cb800511db800c4
:1036a000f485570046000700fe0190003a0007002d
:1036b0008b85e8003e0007008e099000400007005f
:1036c000ee019000340007008b85e8003800070009
:1036d0008e099000400007009e0990001b18b8005a
:1036e000890440000a854800fe019000340007006c
:1036f0008b85e80038000700ee01900030000700dd
:103700008e0990001b18b800890440000a85480003
:103710000a98a30008003a000402420085824a0089
:1037200006034b0087834b0008044c0089844c003f
:103730000a054d008d06e90084827200850273003f
:103740004c3add00850272000100320015002000b5
:10375000443ade001400b2004538de00cb45dd00ff
:103760000b007000c540de00cb4ddd008b8070008b
:103770004549de00cb55dd000b017100c551de006f
:103780000d0378001506070003f0a1000cf0a70058
:1037900003f0a0000c0637001b18b800850240009b
:1037a00006834800e0834b0060044c0007003700ac
:1037b0001b18b8000603400087834800faff370053
:1037c0001b18b8008703400008844800e0844c00c0
:1037d00060054d00000006001b18b80008044000fa
:1037e00089844800faff37000108a300f3053a0076
:1037f0005800be005801be00e3ff37000008a300d8
:10380000ee053a0009047800f9ff37002800fa00b5
:10381000889fbe008a9fbe008c9fbe0003866b00ff
:10382000d50507006400e100440032006408e100af
:103830004a0032006100e100460032006108e10008
:1038400049003200ec0647006000b8003d02be00af
:103850003d03be00f48657006011b8003d04be0071
:103860003d05be007d0320000b0037000000a000d6
:103870008d06e900130032000402420085824a00ee
:1038800006034b0087834b00000040008180480006
:1038900002014900838149000802520089825a00ce
:1038a0000a035b008b835b00f0ff3b0008024200d1
:1038b00089824a000a034b008b834b008d06e90086
:1038c000edff3a008482720086827200f707b20030
:1038d0008782720001003200150020001e04900053
:1038e0003e0b900006035400e63fb0000368a300bf
:1038f000070032000000a7000500a0008301d100ee
:103900000281d3008180d3000080d3000603e80049
:103910008301d1000281d3008180d3000080d300d5
:103920000002eb000482d200ac05070003f0a10006
:103930000cf0a70003f0a000a305370064024700c5
:103940006408e1009d0532003400be003401be0071
:10395000f6ff37006108e100980532006011b800f9
:103960006000b800f1ff370003ff270002002000cd
:10397000fbff37008f1fd100c40507008f87e900c8
:103980000000e000000006001400fa00889fbe005e
:103990008a9fbe008c9fbe000004be000205be00d0
:1039a000680047000a90be000890be00e0050700ce
:1039b0000078a3003d003a006100e1003c003200c5
:1039c0000bf8a3003d003a006400e100380032002b
:1039d0006c0347001e009000f03fb1003602be00ad
:1039e0001603be000008a3000400320004024200d7
:1039f00085824a0006034b0087834b00100798001e
:103a00008e1f78006000b8006011b8005c002000d4
:103a10006d0120006e002000020037008d86e90055
:103a2000fc0020000402420085824a0006034b008d
:103a300087834b0000044000818448000205490050
:103a4000838549006060e1001d60ad0008045200fc
:103a500089845a000a055b008b855b0003003900ee
:103a60001e60ad000802be000a03be000c06e9009d
:103a7000ecff3b000e87e900e8ff3b004f077800b2
:103a800061026000840278008301d1000281d300ca
:103a90008180d3000080d3001e03900041b3de007c
:103aa000f63fb0004d050700470537000b30a0007a
:103ab0000800be000a01be004305370012022000c4
:103ac000825988003d05370023010700b7fd230018
:103ad000b6b72c0065522100e4502e00d6fe370008
:103ae0001e00fa00889fbe008a9fbe008c9fbe0009
:103af0000404be000605be00009fbe000297be0083
:103b0000b2050700040678000800be000a01be00e6
:103b1000ae0507008406780004002000bd050700fc
:103b200005003a008d02b30014002000b90507001b
:103b300001003a00f8866e000802be000a03be00cb
:103b4000f90007003e00be002e01be001e05320037
:103b50000bf0a7000de0a00003f0a7000df0a000ff
:103b60000d08a300d6003a003e02be002e03be00a0
:103b700007f0a10037079800eb0007000df0a60042
:103b8000cf00320001003c000dd0a0008d4f760028
:103b90000a0533006000b8006011b8006260e100ff
:103ba000c9003900d1003e000d28a300d2003a0020
:103bb0000df8a300080032000d58a300d800320011
:103bc0003e02be002e03be00d70007003e00be002e
:103bd0002e01be00c00032003e00be002e01be001d
:103be0006a024700cf050700009fbe000297be0093
:103bf0000df0a7000d30a6000df0a1006d07980094
:103c000067fe2300e6092a00f5672600d4bc2300de
:103c100058ff070009003d003e00be002e01be0017
:103c200014002000dc0507005e029000009fbe002b
:103c30000297be000402e900540798005e0090005d
:103c40006100b9000706070070079800010f98008f
:103c5000120f9800230f98000802be000a03be004e
:103c600075fe0700020607000006be000100e00026
:103c700002003d0060001000e0801800f2ff270005
:103c8000820f5000e08f580083003e000c00be0001
:103c9000f4050700300f9800410f9800520f98006c
:103ca000630f98000800be000a01be00f00507007f
:103cb00040079800f23f2000820f5000e08f58002c
:103cc00005003c0012c02f00f3ff2f00820f5000b0
:103cd000838f58000a003d005e0690000c00e00053
:103ce0000300320001003c000201ea0002067800f5
:103cf0006000b8006011b800400798002700370046
:103d00000800be000a01be00411add004522de00a7
:103d1000f43fb1008400b1003e050700809fbe0063
:103d2000829fbe007e0290008e0a90001e0b9000c3
:103d3000ae0b900040fe07003e0a9000ce0a9000b5
:103d40005e0b9000ee0b90006f0307004f03be0068
:103d50004f02be00809fbe00829fbe000800be00d2
:103d60000a01be00680307007e0290008e0a9000e0
:103d70001e0b9000ae0b90002ffe07004f03be00fd
:103d80004f02be006703070067fe230026e42200ff
:103d9000a5ef2f00f49e230027fe0700809fbe00a2
:103da000829fbe004e0090006100b900ad05070083
:103db00003f0a2000802be000a03be005903070078
:103dc000809fbe00829fbe003e00be002e01be004e
:103dd000610007004f03be004f02be0016fe070041
:103de0004f03be004f02be004e030700ca03070088
:103df000809fbe00829fbe004d000700ce0690004f
:103e00000df0a7008d06ea00090037003e00be0055
:103e10002e01be003e02be002e03be0006fe0700bd
:103e2000009fbe000297be000800be000a01be004f
:103e30003e02be002e03be000d00a700fefd0700df
:103e40000004be000205be008d06d100efff3a005f
:103e50006e02900004e0a600060037000002be00db
:103e60000203be003200070068fe07000004be0027
:103e70000205be004f03be004f02be00eefd07006c
:103e80000c02780044050700ee0690000df0a70034
:103e900003f0a2004c043700ee0690002900070052
:103ea000260007000dd0a7000dc0a0000de0a70060
:103eb0000dc0a2000dc0a60003002000f2ff3700d5
:103ec0001b000700400437000bf8a300020032007b
:103ed0001e000700190007000df8a3003a04320085
:103ee0000d30a70003f0a200370437000bf8a30041
:103ef000f9ff3a00f7ff37003e02be002e03be0076
:103f000009000700eeff320001003c000bf0a200a8
:103f10000a0007000bf0a600030020002a04370067
:103f20000a000700250437000100070091fe370052
:103f300003ff23006000b8000200050003ff270014
:103f4000fcff370020022000010037001002200093
:103f500080598800000006000800fa00889fbe0013
:103f60008a9fbe008c9fbe00980407006420e10079
:103f700015043e006220e100030032008700350096
:103f800003f8a3001004320003f8a30087003a00ee
:103f90000e027800e30407001e0678000004be004d
:103fa0000205be007a000700d7020700009fbe008e
:103fb0000297be000800be000a01be0067fe230093
:103fc000e6092a00f5672600d4bc2300d0020700ca
:103fd000090034003e00be002e01be006c00070048
:103fe000c9020700009fbe000297be000800be0085
:103ff0000a01be00030037000c06e9003e00be00c7
:104000002e01be00620007008bfd07006000070064
:10401000c40207000002be000203be003e00be0054
:104020002e01be00f9fd07000004be000205be001f
:104030000002be000203be007ffd0700009fbe001d
:104040000297be0017042c0006582d0075b62400f8
:10405000f4e02c00b30207003e02be002e03be00b7
:1040600075fd0700370724003608280055a12f00ea
:10407000e4672200ab0207003e02be002e03be0032
:104080006dfd070087082c00e6bf2000d5c0290081
:1040900074072900a3020700809fbe00829fbe0014
:1040a00097fe2b005641240065352b0094d22b003f
:1040b0003e00be002e01be005ffd07000703240086
:1040c000a624260065012200d4fe2a0095020700de
:1040d0003e02be002e03be0057fd070007052c0060
:1040e000f67f2000352b2100a4592b008d020700fc
:1040f0003e02be002e03be004ffd07004f03be0070
:104100004f02be00c1fd0700009fbe000297be0027
:104110000802be000a03be0047fd07000802be00f9
:104120000a03be007f0207000004be000205be00b5
:104130006160b900cb040700009fbe000297be007b
:10414000b7f22b0006012d0015c6250084ca2000f9
:1041500039fd07000802be000a03be007102070015
:104160000004be000205be003e00be002e01be00df
:1041700067fe2300060023006022b8002efd070022
:104180000802be000a03be00660207008e03370065
:1041900007fe23006022b8000600050003ff2f0081
:1041a000020020006000b8008703370010022000e2
:1041b000805988008103370004002000d8043700ac
:1041c0000800fa00889fbe008a9fbe008c9fbe0038
:1041d0000004be000205be00fc0307006220e100ef
:1041e00079033a0003f0a10007ff23000600200036
:1041f0006022b800dffd07000800be000a01be0013
:1042000003f0a100050034000d002800830507001d
:104210000bf0a70003f0a2006b03370067e4230054
:10422000e6092a00f5672600d5bc2300d1fd07006a
:104230000800be000a01be00630335000802be008c
:104240000a03be00fcfc0700009fbe000297be00f0
:1042500017072c0036bc2500951c280024ff2700da
:10426000300207003e02be002e03be00f2fc070033
:10427000170e240076852a00653b220074ec250089
:10428000280207003e02be002e03be00eafc070023
:1042900007142c00e6ac2100e50b28003471260041
:1042a00020020700809fbe00829fbe0097fe2b0069
:1042b000764e2400f5862b00b4812c003e00be0013
:1042c0002e01be00dcfc070047062c0016842700e8
:1042d00055382600a4e42b00120207003e02be005f
:1042e0002e03be00d4fc0700670c2c00265c2900be
:1042f00045692b00044921000a0207003e02be0066
:104300002e03be00ccfc070057112c00369127006d
:104310003565250094412300020207004f03be00cb
:104320004f02be0039fd07003e02be002e03be0054
:10433000c1fc07000802be000a03be00befc070065
:104340000802be000a03be00f60107001e03370084
:104350001400200065053700340020007004370089
:104360000800fa00889fbe008a9fbe008c9fbe0096
:10437000960307006420e10013033e0003f0a10050
:10438000110332000d002000240507000e03370042
:104390000002eb00550537000800fa00889fbe00b8
:1043a0008a9fbe008c9fbe000004be000205be00b6
:1043b00083067800850307006420e100a3003e0027
:1043c000a60032000006eb000bf0a10003ff230063
:1043d000020020006000b8000802be000a03be0010
:1043e000cb01070009003d0003ff2300020020006d
:1043f0006000b8000802be000a03be0003fd07000b
:104400000004be000205be002c00200013fd2300a6
:1044100042612200e1e9250060d52c000802be00bf
:104420000a03be00ba0107001d003d00b3ff2300d0
:10443000a2672b0081852e00a0ca24000802be00be
:104440000a03be00b7010700009fbe000297be002e
:1044500073fe230052cf2600010b2d00509529003a
:104460000802be000a03be0073fc070007ff23001a
:10447000060020006022b800a30107000802be0069
:104480000a03be00a70107003e02be002e03be00c5
:10449000defc07000004be000205be000c06e800ba
:1044a0000800be000a01be0003f0a10067e423007b
:1044b000e6092a00f5672600d4bc23002dfd07007d
:1044c0000800be000a01be004c0035000802be0014
:1044d0000a03be0058fc0700009fbe000297be0002
:1044e000e702240096c42000a5142e0004712c00bd
:1044f0008c0107003e02be002e03be004efc0700ea
:10450000d7042400a6a02c00d5202300743d2a0047
:10451000840107003e02be002e03be0046fc0700d9
:104520005705240026a12800b540200054da2600b3
:104530007c0107003e02be002e03be003efc0700c9
:1045400047042400c687280045cc2b00945a290034
:1045500074010700809fbe00829fbe003e00be0027
:104560002e01be00a7fe2b00a6d72c00159b2d0008
:10457000d47b280030fc070007022c00f6d32f0064
:10458000d5c8250034a62600660107003e02be00fd
:104590002e03be0028fc070047032c00f617280056
:1045a000259e2b00b4cc2b005e0107003e02be000e
:1045b0002e03be0020fc0700b7022c00660a26006e
:1045c0006510250024ce2100560107003e02be00e2
:1045d0002e03be0018fc07004f03be004f02be00b2
:1045e0008afc07000802be000a03be0012fc070096
:1045f0000802be000a03be004a0107000c00e000ea
:104600000f0032000c10a70003f0a20084d122009a
:1046100045442500b61f220097ff23006260e10099
:104620000600320064362700d582230026152c00b0
:1046300007fe23000c10a70007ff23003901070025
:104640000df0a70003f0a2005f0237000330a000c6
:1046500014022000845988005b02370093ff230076
:10466000b21f22004144250080d12200f4ff370010
:104670000800fa00889fbe008a9fbe008c9fbe0083
:104680000004be000205be0003067800cf0207004a
:104690006420e1004c023e00710032006220e10023
:1046a000490239000bf0a1003703240016fc20005a
:1046b000f5312900a49c200003f0a100140107009b
:1046c00067003c0017fe2300a63e2900d5aa27005c
:1046d000b43020000800be000a01be000c01070033
:1046e0000800be000a01be0045003c0067e423004c
:1046f000e6092a00f5672600d4bc23009dfc0700cc
:104700000800be000a01be00520035000802be00cb
:104710000a03be00c8fb0700009fbe000297be0050
:10472000c705240096fa2200b51e2e00a47f2f0094
:10473000fc0007003e02be002e03be00befb0700c9
:10474000170a2400b638270015d02400340f2f0094
:10475000f40007003e02be002e03be00b6fb0700b9
:10476000270b2400c6832e00e57425003469290038
:10477000ec000700809fbe00829fbe003e00be008e
:104780002e01be00e7fe2b0086c22d00b5ef2c00e7
:10479000f4772a00a8fb070087052c0056e72c00b9
:1047a000a51b2a00c4cc2500de0007003e02be0087
:1047b0002e03be00a0fb070097092c00565a2300c9
:1047c000e59b2c0084e12100d60007003e02be00dc
:1047d0002e03be0098fb07004f03be004f02be0031
:1047e0000afc07000802be000a03be0092fb070095
:1047f0000802be000a03be00ca0007001500370009
:104800000802be000a03be00c600070042010700fe
:1048100007ff2300060020006022b800c100070047
:104820000002be000203be0003ff2b0002002000b6
:104830006000b800f5fb070007fe2300060020001b
:104840006022b800b70007000002be000203be00ed
:10485000b40007000cf0a70003f0a200da01370053
:1048600003ff2300020020006000b800f9ff3700ba
:104870000800fa00889fbe008a9fbe008c9fbe0081
:104880000004be000205be00500207006420e100e3
:1048900099003e009500320003f0a100171a240091
:1048a00036582c0005a021000400200031fc070030
:1048b0000800be000a01be00070035009700240072
:1048c000b61f22004544250084d12200b40407000d
:1048d0000004be000205be0047fe230006f32500cb
:1048e00095dc260034882c0053fb070007fe2300cc
:1048f000060020006022b80003f0a70007f0a00027
:1049000088000700da020700801f7800d502070040
:1049100003f0a200009fbe000297be0097ff230095
:10492000060022006022b80043fb07000802be0018
:104930000a03be007b000700809fbe00829fbe006e
:104940003e00be002e01be00f7f3230046542b00ac
:10495000152d2400a446280037fb07004f03be0096
:104960004f02be006f0007000004be000205be003b
:1049700003f0a10067e42300e6092a00f56726009a
:10498000d4bc23006200070004003d0003ff2300a5
:10499000020020006000b800480037000800be0098
:1049a0000a01be000002be000203be0022fb070097
:1049b000009fbe000297be0027ef2b0076ab2b00b6
:1049c00025ea220044722c001bfb0700c7f62300d7
:1049d00026e82000b5632a00f4ad2a005100070044
:1049e0003e02be002e03be0013fb070017fc2b0087
:1049f000562b2100d5542e000490200049000700ba
:104a00003e02be002e03be000bfb07000802be00e4
:104a10000a03be0008fb07000802be000a03be002e
:104a2000400007000004be000205be003e00be00bc
:104a30002e01be0007ea230046772b0065072f00f2
:104a4000948e2700fcfa070047f32b0046f6260059
:104a50009590290014842400320007003e02be0015
:104a60002e03be00f4fa0700a7f92300e67924001c
:104a7000e5172a00941522002a0007003e02be0016
:104a80002e03be00ecfa0700d7fd2b0006eb2d002d
:104a9000b57f2400549d2d00220007003e02be0079
:104aa0002e03be00e4fa070007ff230006002000e3
:104ab00005002000040020001a0007000802be00c4
:104ac0000a03be004f00a6000200370007f0a20054
:104ad000040037000002fd008102fd000203fd001a
:104ae0008303fd0049fb070037013700f3ff270070
:104af000f2ff2f006110b9000330a0001402200063
:104b0000845988003001370007f0a2000500370003
:104b1000809feb005d0107008f87e9000000e00047
:104b2000000006002800fa00889fbe008a9fbe0091
:104b30008c9fbe0007067800878669000c003b004a
:104b4000030478008704780008f0a10009f0a100b0
:104b5000840f5000858f5800860f5900890f5c0024
:104b6000030033000cf0a20001003a000cf0a10099
:104b7000010107006400e1005f0032007801470096
:104b80006408e100610032006c0147007485570041
:104b90003200be001201be003a04be001a05be007b
:104ba0001e039000be0a90008503530006003d00de
:104bb0000004fd008104fd000205fd008305fd00e9
:104bc0008703ea00050378000df8a3000400320013
:104bd00060041400e0841c0060051d00e0851d00d9
:104be0006022b8007d0320000d38e1008006eb0054
:104bf0000b0039004433dd00f300b2008301730081
:104c000039003700848272000d027800e1066400ea
:104c10008b85d1000a85d3008984d3000884d30012
:104c20008703e900f7ff3b00080040008980480047
:104c30000a0149008b81490004003b00600010001c
:104c4000e080180060011900e08119000358a300fa
:104c5000090032008d82720084827200610260005d
:104c60008301d1000281d3008180d3000080d30072
:104c70000603e8001b0037000348a30017003a00b2
:104c80000600e000170034000603e9000d00a30051
:104c900000004800818048000201490083814900ea
:104ca0000348a3000f003a000600e00009003400aa
:104cb0000603e9000000400081804800020149002d
:104cc0008381490001003a000003eb000348a30080
:104cd000f5ff32006022b8000200370084827200c3
:104ce00061826600bd00070003f0a1000cf0a70080
:104cf00003f0a000b4003700640147006408e1003d
:104d000002003a000df8a300ac003a003200be00e9
:104d10001201be00ac0037000800fa00889fbe00f8
:104d20008a9fbe008c9fbe000004be000205be002c
:104d3000260107006420e100a3003e008a00320043
:104d40006708240026e42200a5ef2f00f49e23002c
:104d50006fff07007a003c000800be000a01be0099
:104d600077082c0056382400d5462400341c270030
:104d700000fb0700780035000800be000a01be00f5
:104d800003f0a10007c92300060020000500200051
:104d900004002000f7fa0700710035000800be008b
:104da0000a01be0077ff230076542100b552260089
:104db000e42f280020fa070007fe23000600200049
:104dc0006022b80003f0a70007f0a00055ff07001d
:104dd000a70107000006be00a201070003f0a20021
:104de000009fbe000297be0067fe2300060023005e
:104df0006022b80010fa07000802be000a03be00d5
:104e000048ff0700809fbe00829fbe003e00be009c
:104e10002e01be00b7f22b0006012d0015c625009d
:104e200084ca200004fa07004f03be004f02be00f0
:104e30003cff0700809fbe00829fbe000002be00b4
:104e40000203be00fcf90700009fbe000297be00ef
:104e500017ef2300462a250085f52600c4c12d0042
:104e6000f5f90700c7f72300460e270035fb26009b
:104e7000046e2f002bff07003e02be002e03be0073
:104e8000edf9070007fd23000600200005002000c3
:104e90000400200023ff07004f03be004f02be00a6
:104ea000e5f90700809fbe00829fbe003e00be0065
:104eb0002e01be0007f4230096f92300e5fd26002d
:104ec00094802300dcf90700c7fa2300e6182700c6
:104ed00025142700341b250012ff07003e02be00e8
:104ee0002e03be00d4f9070007fe230006002000b1
:104ef00005002000040020000aff0700ffbb970008
:104f00006fbb9700dfba97004fba9700fefe07000d
:104f10000002be000203be004f01be004f00be00f3
:104f20003afa070007fe2300060020006022b800be
:104f3000fcfe07006102460017010700220037004f
:104f400003ff270022022000825988000001eb00a5
:104f50006000b8001c0037008001eb00f9ff37004b
:104f600003ff2300f9ff370003f8a3001600320007
:104f70008001eb00f5ff3700680447000294be0093
:104f80000094be00fc0447008694be008494be00da
:104f90000900780066000700080078006400070038
:104fa00099007800814f70000b003b000800be00a4
:104fb000ff0207004f00b10003003700f3ff270096
:104fc000f2ff2f006110b9004f06be004f05be0072
:104fd0004f04be000080fa00000006001800200008
:104fe00057002000080453000d003d00060020007b
:104ff00097fc2f000740e1001e00340084827200fd
:10500000610260008301d1000281d3008180d3005e
:105010000080d3000804e800f8ff3a0047002000b1
:105020006104600005047400040464000d00320093
:1050300061004000e080480060014900e0814900d3
:1050400003b8a500070032000603e8006538e10058
:1050500004003a008301d1000281d3008180d30093
:105060000080d300f87f20000830e1000300350005
:10507000080378006000b8006011b8004433dd0018
:10508000f300b2008301730000000600889fbe0099
:105090008a9fbe008c9fbe000404be000605be00b1
:1050a000809fbe00829fbe00480007000406780073
:1050b0000800be000a01be00440007008406780014
:1050c0004f03be004f02be008d4f76007fb09700a9
:1050d00013003300f0ff2f008b8f6b0006003b00a6
:1050e0000d0666000c00a7000a00370007f0a600b6
:1050f000100020000a003700880f5200898f5a00e4
:105100008a0f5b008b8f5b000300390010002000ca
:1051100001003e000000200007f0a7000000ea00a8
:105120004f06be004f05be004f04be000000060043
:10513000800078005002be005003be004439de00fb
:10514000f700b200f37f2000030161000900320084
:105150000218e10016003a00850172008301730015
:10516000838173000008200015003a0040002000f1
:10517000130037008501720083017300838173007f
:1051800005003a0004a8be0006a8be0010002000da
:105190000b0037000201e9000402420085824a0048
:1051a00006034b0087834b000748a300f9ff32003a
:1051b0000740a00004a8be0006a8be0020002000f2
:1051c00080009800920098000000060005ff27006c
:1051d00005826100070032000428e100010032006e
:1051e000240005000600070001003a004400050005
:1051f0000408050002000700f9ff3a00140005004a
:105200006f82610081027000850271008502720068
:10521000000006001400fa00889fbe008a9fbe00ae
:105220008c9fbe0004067800e80247008292be0010
:105230008092be0005007800bdff07006200e1001b
:1052400033003a006000b8006011b8001e039000ff
:105250000c035300f63fb100220035004b03200041
:105260000b30e1002a003d00fb012000faff2f0077
:105270006154b9006c0147008b05d1000a85d30049
:105280008984d3000884d3000603e900faff3b00b9
:105290003200be001201be00000264008182640080
:1052a0000203650083836500050272000602720036
:1052b00007027200160032000884ea008984ea00be
:1052c0000a85ea008b85ea000000640081806400a2
:1052d00002016500838165006022b8001e03900012
:1052e0003eff0700de03900007f0a70003f0a000d8
:1052f0000082eb000400e0008e0290004f06be002a
:105300004f05be004f04be000080fa0000000600fa
:1053100064014700040020003200be001201be00fc
:10532000f4ff37001400fa00889fbe008a9fbe0079
:105330008c9fbe00040678000004be000205be007b
:10534000680047000a90be000890be0078ff070082
:105350006200e1000800be000a01be000400200057
:105360000b003a001e029000e43fb1006e00900076
:10537000fe0090000e0990009e099000f300b2001c
:1053800005fe2300858171000bf0a70003f0a0004b
:10539000040e78000cff37001400fa00889fbe004e
:1053a0008a9fbe008c9fbe00040678000004be00e9
:1053b0000205be00680047000a90be000890be00cb
:1053c0005bff07006200e1000800be000a01be00aa
:1053d00023003a006e009000fe0090000e0990003d
:1053e0009e0990009e02900085024600e47f200006
:1053f0000428e10005003c00d4fc2f000428e10053
:1054000008003d000500200001003700f57f200066
:1054100020022000805988006000b8006011b800a8
:105420000a003700140020000482520007003d00eb
:105430008301d1000281d3008180d3000080d3009a
:105440000402e800faff3a0005002000c42add004b
:10545000f300b200858171000bf0a70003f0a000fb
:10546000d9fe37004f89de0082017800de01370067
:105470001400fa00889fbe008a9fbe008c9fbe0069
:105480000004be000205be00680047000a90be008e
:105490000890be0026ff07000070a7000bf0a100d7
:1054a000304320009e02900080825200b0fe2f0008
:1054b0000028e10011003d00b0fc2f000028e100b1
:1054c000150034001e0990008e0890007e009000a8
:1054d0000501b0000201d1008180d3000080d3001b
:1054e0008502e800fbff3a000b00e000b6fe3b003f
:1054f00060001000e0801800b3fe3700f0ff2f00be
:10550000f1ff27000b00e000affe3b000100280088
:1055100000002000acfe37006000b800aafe370093
:105520000800fa00889fbe008a9fbe008c9fbe00c4
:105530000406780003f0a7000cf0a0000004be00f1
:105540000205be0021ff07006420e100af003e001d
:10555000ab0032000bf0a1000800be000a01be0043
:1055600007ff2300060020006022b80068fd070046
:10557000a3003c000800be000a01be0067e423004f
:10558000e6092a00f5672600d4bc2300f9f80700d5
:105590000800be000a01be007d00350007fe2300a2
:1055a00006002000050020000400200058fd070030
:1055b00008003c000800be000a01be000802be0050
:1055c0000a03be001cf80700009fbe000297be0041
:1055d000160037000c10a20003ff23000200200079
:1055e0006000b8000802be000a03be0046fd0700c6
:1055f00007fe230006002000050020000400200014
:105600000df80700009fbe000297be00def80700fd
:1056100007002c00060020000500200004002000e8
:1056200005f807000004be000205be003e00be00f3
:105630002e01be0077032c00862e2d0095ef26004c
:10564000f461280037fd07003e02be002e03be00b5
:10565000f9f7070027062400c6e72d009565290005
:1056600004c721002ffd07003e02be002e03be002e
:10567000f1f7070077072c00e6dc2d0065c52f0049
:1056800084842a0027fd07003e02be002e03be00d0
:10569000e9f70700a7072400f6242100e50121000f
:1056a00034842b001ffd07003e02be002e03be0007
:1056b000e1f7070047062c00066c2800b5e223003e
:1056c000c47c280017fd0700809fbe00829fbe009b
:1056d00063fe2b00d2bb2400615e2b0050e621004c
:1056e0003e02be002e03be00d3f70700470224008f
:1056f00076e12400c54e26007492230009fd0700c0
:105700003e02be002e03be00cbf7070037042c007c
:10571000c6822d00659a2a00f4a92d0001fd07001c
:105720003e02be002e03be00c3f70700c7042400dc
:1057300076aa2900a5602300a4482d00f9fc0700e3
:105740003e02be002e03be00bbf70700b7032c00cd
:1057500056e52500a5832a0024a62000f1fc0700b9
:105760003e02be002e03be00b3f707004f03be008b
:105770004f02be0025f807000802be000a03be0063
:10578000adf707000802be000a03be00e5fc0700f3
:105790000c00a7000900370097ff2300b61f220066
:1057a0004544250084d122000c10a700ddfc070031
:1057b0000cf0a70003f0a200100037000cf0a700c7
:1057c0000200370003f0a200060037009700240013
:1057d000b61f22004544250084d122000c10a600eb
:1057e0000500370097ff2300b61f2200454425001f
:1057f00084d122000c10a700cafc0700f2fd37007c
:10580000f3ff2700f2ff2f006110b9000330a00062
:105810001402200084598800f8ff3700009fbe0062
:105820000297be006708240026e42200a5ef2f009f
:10583000f49e23004ff80700190034003e00be001c
:105840002e01be0067082400e63c230095fb2800db
:10585000e4872f00aefc07003e00be002e01be0014
:1058600004003c0067fe230006e622006022b80028
:10587000a5fc070028fd0700009fbe000297be00a0
:10588000d7ee23002611200025b02e00642d200025
:1058900069f707003e02be002e03be00a1fc3700e0
:1058a0003e00be002e01be001bfd0700009fbe0093
:1058b0000297be000002be000203be0003ff2300e9
:1058c000020020006000b800d0f7070083816e005e
:1058d0003e02be002e03be0092fc070007fe23001e
:1058e000060020006022b80053f737000800fa00d5
:1058f000889fbe008a9fbe008c9fbe000406780071
:105900000004be000205be0030fe07006420e10076
:105910009f003e009b0032006120e10096003200b3
:1059200003f0a100171b240036582c0005a021000d
:10593000040020000ff807000800be000a01be00a6
:105940000700350097012400b61f220045442500ba
:1059500084d12200920007000004be000205be00b0
:105960008006eb000c00a700cf1ede0003f0a100b4
:105970000bf0a10047fd230006f3250095dc26006f
:1059800034882c002cf707006022b8000003eb00dd
:1059900007fe23000c00a60007ff230061fc0700a0
:1059a000b3fe07000000a7000d00a200adfe070037
:1059b0000c00e00004003a0007fe2300060020006f
:1059c0006022b80050fc070003f0a200009fbe0058
:1059d0000297be0097002400060022006022b80053
:1059e00015f707000802be000a03be004dfc0700c1
:1059f000809fbe00829fbe003e00be002e01be0002
:105a0000f7f4230046542b00152d2400a44628004b
:105a100009f707004f03be004f02be0041fc07001c
:105a20000004be000205be0003f0a10067e42300ed
:105a3000e6092a00f5672600d4bc2300cdf707004d
:105a40000800be000a01be00480035000002be008a
:105a50000203be00f8f60700009fbe000297be00da
:105a600087ce2300f60f28003599260054f92d0023
:105a7000f1f60700a7d62b0006422e0085c02d00a8
:105a8000c499240027fc07003e02be002e03be007e
:105a9000e9f6070067de2300c6232100a58626005d
:105aa00004432d001ffc07003e02be002e03be0073
:105ab000e1f60700a7e52b0056642e00d5b52400bb
:105ac000b40a2c0017fc07003e02be002e03be00e5
:105ad000d9f6070077ec230036de210045522a0074
:105ae00034062f000ffc07003e02be002e03be004e
:105af000d1f60700a7f22b00061a200015a02100fe
:105b0000a4e1230007fc07003e02be002e03be00f6
:105b1000c9f6070017f823001611210015112100fe
:105b2000040b2100fffb07003e02be002e03be0057
:105b3000c1f6070057fc2b0056552500555525008a
:105b400054552500f7fb07003e02be002e03be00a1
:105b5000b9f607000802be000a03be00b6f6070049
:105b60000802be000a03be00eefb07000d00a700fe
:105b700003f0a20014fd37000c00a60003ff230071
:105b800011fd3700f3ff2700f2ff2f006110b9006d
:105b90000330a00014022000845988000afd370059
:105ba000801feb00470007008f87e9000000060018
:105bb000e48240001078a300070032006402400035
:105bc0001178a3003400be001401be0004003200ae
:105bd0000330a700000006003500be001501be001e
:105be0000330a00000000600889fbe0083047800f8
:105bf0000300e0002c00350003003c000082700030
:105c0000040271002600320036432000c500200047
:105c10008383cf000a0039000541b1008283cf00a1
:105c2000070039000541b1008183cf00040039002d
:105c30000541b1008083cf00010039000541b1006a
:105c400085c353006022b800120032000a003b00f6
:105c500084827200610260008301d1000281d3005e
:105c60008180d3000080d3000603e8008743e8006a
:105c7000f7ff3a000700370000004000818048002d
:105c800002014900838149000603e9008743e900d6
:105c9000f9ff3a00d1fc070009f0a70003f0a000cb
:105ca0004f04be000000060060001000e0801800f5
:105cb00060011900e0811900d3ff3b00033e2c0076
:105cc000f7ff37002800fa00889fbe008a9fbe00b9
:105cd0008c9fbe000efe9700a7fc07006108e10044
:105ce0005c0032006200e1005a003e0054003900be
:105cf0006408e100520032006c01470074855700cf
:105d00003200be001201be003a04be001a05be00f9
:105d10009e029000be0e90000d82520017003b00c4
:105d20000402e80046003a00880f5000898f5800ae
:105d30008a0f59008b8f59004100340064014700dd
:105d4000780347003200be001201be003602be00da
:105d50001603be0007f0a10003f0a60007f0a000a4
:105d60000c70a7006ffb070097fc37000000400095
:105d70008180480002014900838149000c00a00095
:105d800008005000898058000a0159008b81590091
:105d900005003b0008004000898048000a014900d6
:105da0008b8149000c00a1000402e900efff3b00d9
:105db00000024000818248000203490083834900b9
:105dc0001b0032000802520089825a000a035b005d
:105dd0008b835b004200f8000500370000004000a4
:105de0008180480002014900838149008d06e90055
:105df0000340a600f9ff37006022b8000d037800c9
:105e000076fc0700780347004200f90008003500df
:105e100002003c000c08a300050032003602be0060
:105e20001603be0007f0a0000c70a7003dfb0700a2
:105e30005e02900004f0a70003f0a20062fc3700ad
:105e40002e009000be0090004e019000de019000f8
:105e50005dfc3700100220000c70a60080598800fd
:105e600056fc3700020ab900001bb9000200b80056
:105e7000810042008100430000000600839f68000b
:105e80000100e00002003d0060001000e08018000a
:105e90000300e00002003d0060011100e0811900f4
:105ea0003c0107004f00e00002003b0060001000d2
:105eb000e080180000000600881f780000047800c9
:105ec0005001be004000be00040040008580480034
:105ed0000601490087814900009cbe000294be0073
:105ee0000400e1000588e1000690e1000798e10068
:105ef00002003100680044001008e8004f047800f8
:105f0000000006001000fa00889fbe008a9fbe00b5
:105f10003004be002005be00c8b79f00d9b79f005f
:105f2000eab79f00fbb79f000404540085845c001f
:105f300006055d0087855d0088bf9f0099bf9f00b3
:105f4000aabf9f00bbbf9f000898be000a98be0072
:105f50008000eb004fb49700dfb497006fb5970057
:105f6000ffb597000440e10005c8e10006d0e1005c
:105f700007d8e10001003100110020001088100056
:105f80004f05be004f04be000080fa00000006006e
:105f90001200fa00889fbe008a9fbe008c1f780006
:105fa0000205be000004be00f4b79f0085bf9f003d
:105fb00096bf9f00a7bf9f000000eb00e0b79f00c7
:105fc000d0b79f00c0b79f00b0b79f00a0b79f0099
:105fd00000067800dfb097006fb097000001400026
:105fe0000000e0000a003d008c00070001003d00b9
:105ff000120020009200070001003d001200200066
:10600000970007007c805700abff070009003700ae
:106010008200070001003d001200200088000700f8
:1060200001003d00120020008d0007007c80570019
:10603000b4ff07006fb297000400e00007003500ce
:1060400010002000010020006011b800080470005a
:10605000898470000a0571008b8571000c06e800c8
:10606000f0032000800f5600daff34000400e00047
:1060700006003d007fb297008fba97001fbb9700c4
:10608000afbb97007c8057008bff07006fa897007d
:106090000000e00004003a002fb49700bfb497005e
:1060a0004fb59700dfb59700890007004f067800cd
:1060b0004f05be004f04be000080fa00000006003d
:1060c000881f780018002000881f7800b0ff0700a4
:1060d0008f87e9004f04780000000600801feb0066
:1060e000abff07008f87e90000000600889fbe0015
:1060f0008a9fbe008c1f78006e00070005003d00df
:106100002f00070007003d003d0007000006eb00e0
:10611000040037003f00070002003d003000070088
:106120001c0020006a000700e5ff07000203be0014
:106130000002be000c00e000010032002800070051
:106140000400be000601be004f0678004f05be00e9
:106150004f04be0000000600889fbe008a9fbe005c
:106160008c1f78005300070003003d001400070057
:1061700006003d00040037002600070003003d0034
:106180006000b8006011b8001d0007005000070053
:10619000d2ff07000203be000002be000c00e000b8
:1061a000010032000e0007000400be000601be0020
:1061b0004f0678004f05be004f04be0000000600e9
:1061c0006000b8006011b8000804500089845800cd
:1061d0000a0559008b8559001c0020000300370078
:1061e0006000b8006011b80005003700e00f5200f1
:1061f000e08f5a00e00f5b00e08f5b0000000600bc
:106200000402500085825800060359008783590014
:10621000000006000006eb00f4ff37004f08de0028
:1062200000007100c0b79f0001804000b0b79f0020
:106230000001eb00afb097000100e0000000060095
:1062400002007000b0b79f0001804000a0b79f001f
:106250000001eb009fb097000100e0000000060085
:1062600002007000a0b79f00018040000fb29700ad
:10627000cf20de000100700090b79f0004024200b2
:10628000130007004f18de000002720084b79f0061
:106290000804440089844c000a054d008b854d009c
:1062a0005fb29700efb297007fb397008fbb970064
:1062b000000006000205be000004be00e00f500012
:1062c000e08f5800e00f5900e08f590000000600f1
:1062d0000800be000a01be0000000600889fbe0044
:1062e0008a9fbe008c1f78000205be000004be001d
:1062f0000006eb00e00f5000e08f5800e00f59005f
:10630000e08f590007003d006000b8006011b80040
:1063100008045000898458000a0559008b855900eb
:106320001c002000e00f5200e08f5a00e00f5b00dd
:10633000e08f5b0002003d000f0007000c00a20090
:106340000800be000a01be00220007000203be00d2
:106350000002be000c00e000010032000600070051
:106360000400be000601be004f0678004f05be00c7
:106370004f04be00000006006000b8006011b800c5
:106380000402500085825800060359008783590093
:10639000000006006022b800060220000000d000c5
:1063a0008180d2000482d2008582d2000000a00049
:1063b0000202520083825a000300310002024200ae
:1063c00083824a000000a1000603e900f3ff3a00bf
:1063d00000000600889fbe008a9fbe008c9fbe0002
:1063e0000404b8000506b8008904460060854e0024
:1063f0000606b8000a054600e0854e000706b8000c
:106400008b054600040eb800890446000a854e003c
:10641000e0854d00050eb8000a0546008b854e004c
:10642000060eb8008b0546000416b8000a054600a3
:106430008b854e000516b8008b054600041eb8007b
:106440008b0546000800be000a01be004f06be00d4
:106450004f05be004f04be00000006000400fa0015
:10646000000f7800110798000000eb00000888007a
:106470001e009000100888001e0078002008880088
:106480000080fa00000006000000fa002200200050
:1064900061042000700520002374200081497800e9
:1064a00080497800824978000000eb003031880094
:1064b000716220009140780000c8b30000c0600005
:1064c0000004e0000600320027c6bf000042b20010
:1064d0000004e00001003a006400070027e6a9007c
:1064e00027a6a9000080fa00000006001200fa00aa
:1064f000000f980031318000f0cf2f000080600045
:1065000030318800313180000010200000807000a0
:106510003031880020318000200798002031800031
:106520003007980031318000f0cf2f0000806000ec
:106530003031880031318000001020000080700070
:106540003031880021318000680047002100980028
:10655000213180006800470031009800ee40900033
:10656000680047006040900080cf5000e1ff3a0093
:10657000ce4090000e08900031409800fe40900000
:106580000e08900021409800ee4090000e08900008
:10659000114098000080fa00000006001200fa0086
:1065a000000f980031318000f0cf2f000080600094
:1065b00030318800313180000030200000807000d0
:1065c0003031880020318000000f780020318000b9
:1065d000100798002031800020079800313180009a
:1065e000f0cf2f0000806000303188003131800012
:1065f00000302000008070003031880021318000a0
:1066000068004700010878002131800068004700d9
:106610001100980021318000680047002100980097
:10662000ae409000680047002040900080cf5000ae
:10663000dcff3a00ae4090000e0890001140980038
:10664000be4090000e08900021409800de4090006f
:106650000e089000014878009e4078000e089000d7
:10666000314098000080fa00000006000800fa009f
:1066700042c0bf000080fb004500de00604798007c
:106680009002800010079800ff3ffc0021042000ca
:106690009140780000ceb30000c0700042e0b70027
:1066a0001e009000900288005005200020079800ee
:1066b0002e009000303b8800a00a200020079800a0
:1066c0002e009000303b880027a6a8009002800092
:1066d000000f7800ff3ffc006e40900067406000b4
:1066e000c500dd0042c0bf007f4060000140700077
:1066f00042e0b7001e007800900288000080fa0097
:10670000000006001800fa00100f9800210f9800f2
:106710000000eb00200798001e0890002040900029
:10672000ec4f500011003e001e08900020409000e9
:106730000004e0000d0032001e08900010409000a0
:10674000ff4f500009003e001e08900010409000ce
:106750000004e000050032001e089000b0409000e8
:1067600030c6b30080cf5000030036000000eb00bd
:10677000300f9800770037001e089000b04090005e
:1067800070004700014878001e089000904090007b
:106790006e004700014878001e089000a04090005d
:1067a0006e004700114098002e0890000000e000a5
:1067b0000e00320042c0bf000080fb004500de003a
:1067c000204f98009002800010079800ff3ffc00c7
:1067d000210420009140780000ceb30000c070007a
:1067e00042e0b7001e0090009002880027c6bf005c
:1067f0000080fb004500de00614060000080fb007f
:10680000400798004e0090000000e00001003a00b0
:1068100096ff070027c6bf000080fb004700de0090
:106820000080fb00300798003e0090000000e00070
:106830000600320023c6bf000080fb004700de00d8
:106840000080fb002007980027e6a9003131800076
:10685000f0cf2f000080600030318800313180009f
:10686000001020000080700030318800213180004d
:106870006c004700010878001e08900090407800e6
:106880006c0047001140980031318000f0cf2f009c
:1068900000806000303188003131800000302000fd
:1068a00000807000303188007000470010007800d0
:1068b000203188006e0047001000780020318800e9
:1068c0006c00470010007800203188003e009000e6
:1068d0000000e0000a00320027e6a8002e00900029
:1068e0000000e0000100320023e6a8004e00900006
:1068f0000000e000060032005cff070004003700e3
:106900004e0090000000e00001003a0027a6a90018
:106910002e0890000000e0000c0032009002800081
:10692000000f7800ff3ffc002e4890006740600099
:10693000c500dd0042c0bf007f4060000140700024
:1069400042e0b7001e00780090028800100020008e
:10695000300f98003e0890000080fa00000006000a
:106960001600fa00000f9800110f98000000eb00cd
:10697000200798000e089000a0409000b0c3b3001c
:1069800080cf500009003e000e089000904090001b
:10699000b0c3b30080cf500004003e000e0890004a
:1069a00030409000f84f5000030036000000eb002c
:1069b000200f9800700037000e089000a040900053
:1069c0006e004700114098000e0890009040900023
:1069d0006e004700014878001e0890000000e000ab
:1069e0000e00320042c0bf000080fb004500de0008
:1069f000204f98009002800010079800ff3ffc0095
:106a0000210420009140780000ceb30000c0700047
:106a100042e0b7001e0090009002880027c6bf0029
:106a20000080fb004500de00614060000080fb004c
:106a3000400798004e0090000000e00001003a007e
:106a40000aff070027c6bf000080fb004700de00ea
:106a50000080fb00300798003e0090000000e0003e
:106a60000600320023c6bf000080fb004700de00a6
:106a70000080fb002007980027e6a9003131800044
:106a8000f0cf2f000080600030318800313180006d
:106a9000001020000080700030318800213180001b
:106aa0006c004700010878000e089000b04090008c
:106ab0006c0047000148780031318000f0cf2f0092
:106ac00000806000303188003131800000102000eb
:106ad00000807000303188006c00470010007800a2
:106ae000203188006e0047001000780020318800b7
:106af0003e0090000000e0000a00320027e6a800f7
:106b00002e0090000000e0000100320023e6a80003
:106b10004e0090000000e00006003200d3fe0700a7
:106b2000040037004e0090000000e00001003a0031
:106b300027a6a9001e0890000000e0000c0032000b
:106b400090028000000f7800ff3ffc002e4890006c
:106b500067406000c500dd0042c0bf007f406000ac
:106b60000140700042e0b7001e00780090028800eb
:106b700010002000200f98002e0890000080fa00de
:106b8000000006000600fa00200798001000200010
:106b9000000f78000b0037000000eb001007980092
:106ba000030037001e0090000000e8001007980066
:106bb0009e0090002e009000808f5000f9ff35005d
:106bc0001e0fe800e00020009e0f1000f2ff3400ce
:106bd0000080fa00000006000000fa004507a80047
:106be0004527a8004547a9000080fa0000000600dc
:106bf0000000fa004507a8004527a9004547a9005d
:106c00000080fa00000006000000fa004507a80016
:106c10004527a9004547a8000080fa0000000600ab
:106c20000000fa004507a9004527a8004547a8002d
:106c30000080fa00000006000000fa004507a800e6
:106c40004527a8004547a8000080fa00000006007c
:106c50000000fa00201680000030a00020168800f6
:106c60002116800070ff2f00008060002016880031
:106c70000080fa00000006000200fa00004f7800d1
:106c80009116800000f02f00808060001e00fb0045
:106c900000804000901688000080fa000000060086
:106ca0000200fa00004f78009116800000f02f00db
:106cb000808060001e80fb000080400090168800ed
:106cc000e3ff07000080fa00000006000000fa0061
:106cd00020168000b1ff2f00010060002016880000
:106ce00010c0b300eeff07000080fa0000000600ad
:106cf0000200fa00000f7800201680000020a0009b
:106d000020168800040037001e007800104078002c
:106d10001e0fe800e2ff07001e0078001040780018
:106d20000004e000f8ff3a000080fa0000000600ce
:106d30000200fa00004f780021168000b0ff2f00fb
:106d400000806000201688009e40780000c8b300d4
:106d500000c04000d2ff07000080fa0000000600db
:106d60000000fa0021168000001020000080700052
:106d7000201688002003200082ff070021168000d3
:106d8000b0ff2f0000806000201688004001200026
:106d90007cff0700f0c0b300c1ff070040012000e6
:106da00078ff070010c0b300bdff070040012000be
:106db00074ff070080c3b300b9ff07000080fa002a
:106dc000000006000400fa00100798009e009000e2
:106dd00000942000cce507000040eb00d4ff070042
:106de0001e009000c2ff07001e009000cee50700c5
:106df000000f78000300370000c2b300a8ff0700af
:106e00001e0fe800f00020009e0f1000faff340073
:106e10000080fa00000006000400fa001007980045
:106e20009e00900010952000b7e5070080c2b300d7
:106e3000bfff07001e009000adff07001e0090007e
:106e4000b9e50700000f78000300370000c2b30067
:106e500093ff07001e0fe800f00020009e0f1000b7
:106e6000faff34000080fa00000006000000fa007b
:106e7000048320006000b8006011b800009abe00d2
:106e80000292be00848320006000b8006011b80048
:106e9000009abe000292be00048420006000b80088
:106ea0006011b800009abe000292be0084842000e7
:106eb0006000b8006011b800009abe000292be00e7
:106ec000048520006000b8006011b800009abe0080
:106ed0000292be00848520006000b8006011b800f6
:106ee000009abe000292be00048620006000b80036
:106ef0006011b800009abe000292be008486200095
:106f00006000b8006011b800009abe000292be0096
:106f1000048720006000b8006011b800009abe002d
:106f20000292be00848720006000b8006011b800a3
:106f3000009abe000292be00048820006000b800e3
:106f40006011b800009abe000292be008488200042
:106f50006000b8006011b800009abe000292be0046
:106f6000048920006000b8006011b800009abe00db
:106f70000292be00848920006000b8006011b80051
:106f8000009abe000292be00048a20006000b80091
:106f90006011b800009abe000292be00848a2000f0
:106fa0006000b8006011b800009abe000292be00f6
:106fb0000000eb00804588000000eb009045880051
:106fc0000000eb00a04588000000eb00b045880001
:106fd0000000eb00c04588000000eb00d0458800b1
:106fe0000000eb00e04588000000eb00f045880061
:106ff0000000eb00004688000000eb00104688000f
:107000000000eb00204688000000eb0030468800be
:107010000000eb00404688000000eb00504688006e
:107020000080fa00000006000400fa00004f78001b
:1070300010c1b3009e4f100003003a001000200062
:10704000100798003800370020c1b3009e4f100091
:1070500003003a002000200010079800320037009b
:1070600030c1b3009e4f100003003a0030002000f2
:10707000100798002c003700a0c0b3009e4f1000ee
:1070800003003a0040002000100798002600370057
:10709000b0c0b3009e4f100003003a005000200023
:1070a0001007980020003700c0c0b3009e4f1000aa
:1070b00003003a0060002000100798001a00370013
:1070c00030c0b3009e4f100003003a007000200053
:1070d000100798001400370040c0b3009e4f100006
:1070e00003003a0080002000100798000e003700cf
:1070f00050c0b3009e4f100003003a0090002000e3
:10710000100798000800370000c1b3009e4f100020
:1071100003003a000000eb0010079800020037005f
:107120000000eb00100798001e0090000080fa009d
:10713000000006000000fa00c922a8000080fa0042
:10714000000006000000fa00c922a9000080fa0031
:10715000000006000000fa00601680000110200008
:1071600001007000601688000080fa000000060030
:107170000000fa0060168000f1ef2f0001006000af
:10718000601688000080fa00000006000200fa0085
:10719000e8ff07000040eb00004f780010003700c8
:1071a000ecff0700cbc2bf00624060000004e000bb
:1071b000060032001e4090000080fb0000004000ee
:1071c0000004a00010479800030037001e40900004
:1071d0000040400010479800e5ff07001e4fe80000
:1071e00070c0b3009e4f1000edff36001e409000af
:1071f0000080fb000080fa00000006000400fa0096
:10720000204798000040eb00004f78000c0037004a
:107210002e4090000004e00002003d00c5ff070082
:1072200001003700c7ff0700caff0700d0ff0700b3
:107230002e40900000404000204798001e4fe8007c
:1072400070c0b3009e4f1000f1ff3600b9ff070079
:107250000080fa00000006000000fa00b5ff0700f9
:10726000bcff0700c2ff07000080fa000000060014
:107270000000fa00b3ff0700b6ff0700bcff0700dd
:10728000acff07000080fa00000006000000fa00d2
:10729000b7ff0700a7ff0700aeff0700a9ff070021
:1072a000b3ff07000080fa00000006000000fa00ab
:1072b000afff0700a3ff0700a6ff07009dff070021
:1072c0000080fa00000006000400fa00000f7800b9
:1072d000214798009460a900ecff070000cab300a2
:1072e000c6ff0700dcff07001e0078004800de0034
:1072f000c2ff0700d8ff07001e007800bfff07008d
:10730000d5ff07002e409000bcff0700d2ff07000a
:10731000e6ff0700f00020001afe07009460a800b6
:107320000080fa00000006000400fa001007980030
:107330009460a900d5ff070000cab300afff0700a3
:10734000c5ff07001e0090004800de00abff0700ed
:10735000c1ff07001e009000a8ff0700beff070046
:10736000caff070010cab300a4ff0700baff070056
:1073700086ff0700004f7800ccff07009460a8004c
:107380001e80fb000080fa00000006000400fa00e6
:10739000404b80000000e00003003a000000eb00da
:1073a0001007980010003700604b8000deff0700d8
:1073b0000080fb00000f78001e00e00005003a008e
:1073c0000000eb00404b88000000eb001007980025
:1073d00005003700604b80000000e800604b88002b
:1073e0001e007800100798001e0090000080fa0030
:1073f000000006000200fa00004f7800404b8000b9
:10740000e10f50001300320070c1b3009e4f100016
:107410000a003a00604b80008040eb00aaff0700a2
:107420000000eb00504b8800e0532e0065fe070083
:10743000007d2000d3fd070006003700604b800070
:107440009e407800a0ff0700604b80000000e8002d
:10745000604b88000080fa00000006000400fa007b
:10746000caff0700000f78001e00e0000300320092
:107470001e0078001007980019013700c942a800c3
:10748000c962a800c982a800c9a2a800c142a80078
:10749000c0e2a800c9c2a8000000eb00000f7800fd
:1074a000c942a900b12c20009140780000c8b30067
:1074b00000c060000004e00002003a00100020005c
:1074c000000f7800cbc2bf0001c8b30001406000cc
:1074d0000004e00002003a0010002000000f7800d5
:1074e000c2c2bf00614060000004e00002003a0038
:1074f00080002000000f7800d3c2bf00624060000f
:107500000004e00002003a00f0002000000f7800c4
:10751000c2c2bf00624060000004e00002003a0006
:1075200060012000000f7800c942a800c962a900cc
:10753000cbc2bf0001c8b300014060000004e000fe
:1075400002003a0020002000000f7800cbc2bf00ec
:1075500001c8b300014060000004e00002003a00ee
:1075600020002000000f7800c2c2bf006140600010
:107570000004e00002003a0090002000000f7800b4
:10758000d3c2bf00624060000004e00002003a0085
:1075900000012000000f7800c2c2bf0062406000fe
:1075a0000004e00002003a0070012000000f7800a3
:1075b000c962a800c982a900cbc2bf0001c8b3003c
:1075c000014060000004e00002003a0030002000aa
:1075d000000f7800cbc2bf0001c8b30001406000bb
:1075e0000004e00002003a0030002000000f7800a4
:1075f000c2c2bf00614060000004e00002003a0027
:10760000a0002000000f7800d3c2bf0062406000dd
:107610000004e00002003a0010012000000f780092
:10762000c982a800c9a2a900cbc2bf0001c8b3008b
:10763000014060000004e00002003a004000200029
:10764000000f7800cbc2bf0001c8b300014060004a
:107650000004e00002003a0040002000000f780023
:10766000c2c2bf00614060000004e00002003a00b6
:10767000b0002000000f7800d3c2bf00624060005d
:107680000004e00002003a0020012000000f780012
:10769000c9a2a800c142a900cbc2bf0001c8b30063
:1076a000014060000004e00002003a0050002000a9
:1076b000000f7800cbc2bf0001c8b30001406000da
:1076c0000004e00002003a0050002000000f7800a3
:1076d000c2c2bf00614060000004e00002003a0046
:1076e000c0002000000f7800d3c2bf0062406000dd
:1076f0000004e00002003a0030012000000f780092
:10770000c142a800c0e2a900cbc2bf0001c8b300bb
:10771000014060000004e00002003a006000200028
:10772000000f7800cbc2bf0001c8b3000140600069
:107730000004e00002003a0060002000000f780022
:10774000c2c2bf00614060000004e00002003a00d5
:10775000d0002000000f7800d3c2bf00624060005c
:107760000004e00002003a0040012000000f780011
:10777000c2c2bf00624060000004e00002003a00a4
:1077800080012000000f7800c0e2a800c9c2a90053
:10779000cbc2bf0001c8b300014060000004e0009c
:1077a00002003a0070002000000f7800cbc2bf003a
:1077b00001c8b300014060000004e00002003a008c
:1077c00070002000000f7800c2c2bf00614060005e
:1077d0000004e00002003a00e0002000000f780002
:1077e000d3c2bf00624060000004e00002003a0023
:1077f00050012000000f7800c2c2bf00624060004c
:107800000004e00002003a0090012000000f780020
:10781000c9c2a8001e00e0002f0032000000eb00eb
:107820000008880060092000d6fc0700c942a900b2
:10783000c962a900c982a900c9a2a900c142a900c0
:10784000c0e2a900c9c2a90000003700cbc2bf0036
:1078500001c8b300014060000004e000fbff3200fb
:10786000c2c2bf00614060000004e000f7ff3200c8
:10787000d3c2bf00624060000004e000f3ff3200aa
:10788000c2c2bf00624060000004e000efff3200af
:10789000c942a800c962a800c982a800c9a2a8005c
:1078a000c142a800c0e2a800c9c2a800504b800095
:1078b0000000e000080032001e007800cdfe070046
:1078c000700120009e0f100003003a000000eb0042
:1078d00010079800020037001e007800100798007b
:1078e0001e0090000080fa00000006000800fa0068
:1078f000009fbe000297be0004202c0035a6210088
:10790000c65d2a00c70424003e00be002e01be0052
:1079100049ef07000080fa00000006000800fa00a6
:10792000009fbe000297be0014d1220045442500ee
:10793000b61f2200970024003e00be002e01be00ac
:107940003def07006022b80006002800670624000b
:10795000aeef07000080fa00000006000000fa0009
:1079600000408000e10f500008003a0008c8bf0046
:10797000e14f500003003a00e0542e0026fd0700be
:1079800002003700e0552e0023fd07000080fa00ba
:10799000000006000800fa00230207003402070076
:1079a000304b8000e10f500005003a00a08120001c
:1079b00004fd07009080200017fd07007c003700c1
:1079c000804580006101b9000080eb008080eb0001
:1079d0000201400083814800220798003307980085
:1079e000f0002000010020002e019000be01900058
:1079f000800f5100818f590031003e002e00900011
:107a0000be009000006001000f0037001100370039
:107a10001300370015003700290037002800370011
:107a200027003700260037002500370024003700e4
:107a300014003700160037000f003700170037001a
:107a4000190037001b003700b0c2b3002047980070
:107a50001d003700d0c2b300204798001a0037003d
:107a600080c7b3002047980017003700f0c2b3006a
:107a70002047980014003700c0c7b3002047980083
:107a80001100370000c5b300204798000e003700f2
:107a900030c4b300204798000b003700e0c5b300a6
:107aa0002047980008003700e0c3b3002047980043
:107ab00005003700c0c3b30020479800020037001c
:107ac00000c2b300204798000000eb00000f7800d0
:107ad0000c0037009e007800a0812000008040004c
:107ae000104078000004e00005003a009e00780095
:107af000a08120008080400000c2b3008048780050
:107b00001e0fe800f10020009e8f1000f1ff3600ec
:107b10002e40900029e8b7000040eb002ae8b700ab
:107b2000a04580000000e0000400320080c2b300e5
:107b300027e8b70010c3b30028e8b700c0458000ad
:107b40000000e0000200320020c3b30028e8b700c4
:107b5000e04580000000e0000200320030c3b300c6
:107b600028e8b700004680000000e0000200320074
:107b700040c3b30028e8b700204680000000e000c2
:107b80000200320050c3b30028e8b700404680002e
:107b90000000e0000200320060c3b30028e8b70034
:107ba000a081200087fc0700908020009afc07003d
:107bb0000080fa00000006000400fa00000f7800c0
:107bc0001e007800100798001e009000e30f500080
:107bd000300032001e009000e30f500007003c0010
:107be0001e009000e10f50000e0032001e009000b9
:107bf000e20f500019003200640037001e009000b0
:107c0000e50f5000490032001e009000e50f5000c3
:107c10003b0035001e009000e60f5000510032007e
:107c20005a00370070010700008320003002be00b8
:107c30002003be006000b8000200200003ff230004
:107c4000f2ee070004832000009abe000292be00fc
:107c500050ff0700980107004c0037006201070041
:107c6000008320005001be004000be0004832000bd
:107c70005403be004402be006fee070004832000e0
:107c8000009abe000292be0042ff07008a01070070
:107c90003e00370054010700008320005001be0061
:107ca0004000be006022b8006033b80031ef07002a
:107cb0000000e000010035000700370004832000c9
:107cc0006000b8000200200053042400009abe00a7
:107cd0000292be0007003700008320005001be0062
:107ce0004000be0028ef070004832000009abe0079
:107cf0000292be0027ff07006f0107002300370034
:107d000039010700008320005001be004000be0082
:107d10006def070004832000009abe000292be00af
:107d20001cff070064010700180037002e01070040
:107d3000008320003002be002003be006000b800b7
:107d4000020020004302240065ef070004832000a6
:107d5000009abe000292be000eff07005601070007
:107d60000a00370020010700008320005001be00f8
:107d70004000be0078f0070004832000009abe0097
:107d80000292be0003ff07004b0107000080fa00cb
:107d9000000006000400fa00000f78001e007800c2
:107da000100798001e009000e30f50008e00320074
:107db0001e009000e30f500007003c001e009000e2
:107dc000e10f50000e0032001e009000e20f500044
:107dd00048003200d40037001e009000e50f50002c
:107de000c30032001e009000e50f5000bb003500bc
:107df0001e009000e60f5000c2003200ca0037009b
:107e0000f900070006c8bf00e14f500011003a001a
:107e1000008320005001be004000be00e6f00700d5
:107e200004832000009abe000292be0008c8bf0072
:107e3000e14f500007003a00008320005001be00cf
:107e40004000be00a9fe070004832000009abe0087
:107e50000292be0007c8bf00e14f500007003a0081
:107e6000008320005001be004000be00d4f0070097
:107e700004832000009abe000292be0006c8bf0024
:107e80000004e00014003a0007c8bf000004e0004e
:107e900011003a0008c8bf00e14f500007003a0047
:107ea000008320005001be004000be009bfe070082
:107eb00004832000009abe000292be0000832000ce
:107ec0005001be004000be0021f1070004832000e5
:107ed000009abe000292be000040eb0006e8b70028
:107ee0000040eb0007e8b700aafe0700f200070019
:107ef0008d003700bc00070006c8bf00e14f5000ee
:107f000011003a00008320005001be004000be0076
:107f100011f1070004832000009abe000292be0007
:107f200008c8bf00e14f500007003a00008320005e
:107f30005001be004000be006cfe0700048320001c
:107f4000009abe000292be0007c8bf00e14f500079
:107f500007003a00008320005001be004000be0030
:107f6000fff0070004832000009abe000292be00ca
:107f700006c8bf000004e00014003a0007c8bf00b4
:107f80000004e00011003a0008c8bf00e14f5000b3
:107f900007003a00008320005001be004000be00f0
:107fa0005efe070004832000009abe000292be001d
:107fb000008320005001be004000be00f4f0070026
:107fc00004832000009abe000292be000040eb0035
:107fd00006e8b7000040eb0007e8b7006dfe0700b9
:107fe000b5000700500037007f00070006c8bf003b
:107ff000e14f500011003a00008320005001be0004
:108000004000be00e4f0070004832000009abe0098
:108010000292be0008c8bf00e14f500007003a00be
:10802000008320005001be004000be002ffe07006c
:1080300004832000009abe000292be0007c8bf0061
:10804000e14f500007003a00008320005001be00bd
:108050004000be0086f1070004832000009abe00a5
:108060000292be0006c8bf000004e00014003a00ff
:1080700007c8bf000004e00011003a0008c8bf00b4
:10808000e14f500007003a00008320005001be007d
:108090004000be0021fe070004832000009abe00bd
:1080a0000292be00008320005001be004000be00ce
:1080b000eff1070004832000009abe000292be0088
:1080c0000040eb0006e8b7000040eb0007e8b7000f
:1080d00030fe0700780007001300370010c0b3001f
:1080e00006e8b700e0562e004bfb07000e003700f5
:1080f00010c0b30007e8b70070572e0046fb07001a
:108100000900370008c8bf00e14f500003003a00e3
:108110000040eb0008e8b7000200370010c0b300d1
:1081200008e8b7000dfe07000080fa000000060016
:108130001000fa0040079800510798006207980065
:10814000730798006000b8000200200003ff2300be
:10815000009fbe000297be00150037004e0290003f
:10816000de0290006e039000fe0390003e00be0011
:108170002e01be0030ed0700009fbe000297be003a
:108180006022b8000600200007ff23004e00900088
:10819000de0090006e019000fe0190005af2070090
:1081a00040079800510798006207980073079800ed
:1081b0006022b8000600200007ff23004e00900058
:1081c000de0090006e019000fe01900050f207006a
:1081d0000000e000e1ff3d003e00be002e01be00b9
:1081e0000080fa00000006000000fa002bc8bf0063
:1081f0000004e0000a003a006011b8008000eb00c3
:1082000090802000cfe0070004832000009abe0089
:108210000292be003100070010c0b3002be8b70087
:108220000080fa00000006000000fa0030582e001e
:108230009180200010000900b05878001001b100b2
:10824000008320005001be004000be00809fbe00a1
:10825000829fbe0040592e00801f78009080200031
:1082600075e10700ea8757000080fa000000060069
:108270000000fa0030582e00a181200010000900f3
:10828000b05878001001b100808320005001be007a
:108290004000be00809fbe00829fbe0090592e000d
:1082a000801f7800a081200063e10700ea87570063
:1082b0000080fa00000006000000fa000040eb0019
:1082c0002ce8b700a0812000befa070090802000b3
:1082d000d1fa07000080fa00000006000000fa0052
:1082e00010c0b3002be8b7000040eb0003e8b70074
:1082f0000040eb0004e8b7000040eb0005e8b700e1
:108300000040eb0002e8b7000000eb00704188007d
:108310000080fa00000006000c00fa00e0592e0070
:10832000a8fa07004dfc0700204798002e40900057
:108330000004e000fbff32002e409000f84f500098
:108340005c003a00f05a2e009efa070043fc07003a
:10835000204798002e4090000004e000fbff320010
:108360002e4090000000fb006101b900d0ff2f00fb
:10837000f1ff2f000201400083814800220798008e
:108380003307980000012000010020002e0190001a
:10839000be019000800f5100818f590032003e00d5
:1083a0002e009000be009000006001002500370004
:1083b00027003700290037002b0037002a0037003c
:1083c0002900370028003700150037001700370054
:1083d000190037002400370023003700220037003f
:1083e0000300370005003700070037000900370099
:1083f0000000eb00000f78001d0037001000200087
:10840000000f78001a00370020002000000f7800cd
:108410001700370030002000000f780014003700ec
:1084200040002000000f78001100370050002000ad
:10843000000f78000e00370060002000000f780069
:108440000b00370070002000000f78000800370094
:1084500080002000000f7800050037009000200009
:10846000000f780002003700a0002000000f780005
:10847000a10020009e8f1000640032001e027800d0
:10848000008320005001be004000be00e58c2000ab
:108490004322dd0005024200009abe000292be00a7
:1084a000005c2e0047fa070040062000b5f90700df
:1084b000560037002e4090000000fb006101b9001b
:1084c000d0ff2f00f1ff2f00020140008381480000
:1084d0004207980053079800000120000100200087
:1084e0004e019000de019000800f5100818f5900f5
:1084f00032003e004e009000de009000006001005f
:108500002500370027003700290037002b003700ef
:108510002a003700290037002800370015003700ef
:1085200017003700190037002400370023003700f8
:10853000220037000300370005003700070037002e
:10854000090037000000eb00000f78001d00370025
:1085500010002000000f78001a00370020002000d3
:10856000000f78001700370030002000000f78005f
:108570001400370040002000000f78001100370081
:1085800050002000000f78000e003700600020002f
:10859000000f78000b00370070002000000f7800fb
:1085a0000800370080002000000f78000500370029
:1085b00090002000000f780002003700a00020008b
:1085c000000f7800a10020009e8f10000f003200e5
:1085d0001e007800c300dd00e08c20000080400019
:1085e0005001be004000be0004832000009abe007f
:1085f0000292be0010c0b3002be8b700105d2e0041
:10860000f0f90700400620005ef907000080fa003c
:10861000000006000400fa00881f78002cc8bf0084
:108620000004e00082003a0002c8bf00e14f5000a1
:1086300046003a000000eb00100798000000eb0035
:10864000000f78000a0037009e007800908020001c
:10865000008040009040780050c6b30080cf5000aa
:1086600002003a001e007800100798001e0fe80074
:108670001e04780090802000abdf0700800f5400bc
:10868000f1ff390005c8bf00e14f500014003a0067
:108690001e009000000fe800090037001e0178005e
:1086a0009e00e8009080200000804000904078000c
:1086b0009080200000004100014878001e0fe80073
:1086c0001e0478009080200097df0700800f540080
:1086d000f2ff39000040eb0005e8b7001800370052
:1086e0009080200090df0700000f7800090037001d
:1086f0001e01e8009e00780090802000008040006d
:1087000090407800908020000000410001487800ef
:108710001e0fe9001e0090009e0f1000f4ff3c00a9
:108720001e0090008000e8009080200080804000c3
:10873000d0c2b3008048780010c0b30005e8b7008d
:1087400090802000b4f90700350037002bc8bf0027
:10875000e14f500007003a00704180000000e00047
:1087600002003a000040eb0009e8b7000000eb000f
:108770007041880004c8bf00e14f500014003a0067
:108780000040eb0004e8b7000000eb00000f7800a9
:10879000090037001e0178009e00e800908020004c
:1087a0000080400090407800908020000000410050
:1087b000014878001e0fe8001e0478009080200019
:1087c00059df0700800f5400f2ff39001400370012
:1087d00010c0b30004e8b7009080200052df07000b
:1087e0000000e800000f7800090037001e01780043
:1087f0009e00e900908020000080400090407800ba
:108800009080200000004100014878001e0fe90020
:108810001e00e000f5ff3c00d0c2b30009e8b7003d
:108820000040eb002be8b700908020007af90700a9
:108830004f0478000080fa00000006001600fa00dd
:10884000205e2e005ff90700005f2e0072f907001e
:1088500002fb0700404798004e4090000004e000f3
:10886000fbff32004e409000e74f500038003200ce
:108870004e409000ecf907006a00b900100798001c
:10888000f6fa0700404798004e4090000004e000d0
:10889000fbff32004e409000e3f9070080007800b3
:1088a0001e00900001004000100798009e009000fc
:1088b000b0032000808f500002003600b00320007b
:1088c000100798001e0090004a00dd007000400074
:1088d000604b8800e50047001e009000801f780074
:1088e00000602e00801f780001007800d2df0700b2
:1088f000e48757000000eb00000f78000900370004
:108900009e00780065004700614078008040780054
:10891000604b80001e004000700050006afa0700a3
:108920001e0fe800e00020009e0f1000f4ff36004c
:1089300010002000504b88006500470021f9070017
:10894000c0602e0034f90700803e20008df807003b
:108950000080fa00000006001600fa00881f780068
:10896000c0612e0017f90700005f2e002af90700ea
:10897000bafa0700404798004e4090000004e0001b
:10898000fbff32004e409000e74f500033003200b2
:108990004e409000a4f907006a00b9001007980043
:1089a000aefa0700404798004e4090000004e000f7
:1089b000fbff32004e4090009bf9070080007800da
:1089c0001e00900001004000100798009e009000db
:1089d000b0032000808f500002003600b00320005a
:1089e000100798001e0090004a00dd007000400053
:1089f000604b88000000eb00000f78000900370092
:108a00001e047800604b80001e0040007000500083
:108a100045fa07008040780065004700017478003f
:108a20001e0fe800e00020009e0f1000f4ff36004b
:108a3000e50047000040eb00805098001000200047
:108a4000404b880065004700def80700b0622e004a
:108a5000f1f80700803e20004af807004f04780034
:108a60000080fa00000006000000fa002cc8bf00d9
:108a7000e14f500015003a00004080000000e8007f
:108a80000040880000408000e30f500002003400e6
:108a90000000eb0000408800004080007100b90039
:108aa000800078006097200000804000c5f8070033
:108ab000004080007100b90080007800a09b200079
:108ac00000804000d4f807000e00370010c0b3004b
:108ad0002ce8b700004080007100b90080007800e9
:108ae0006097200000804000b6f80700004080003a
:108af0007100b90080007800a09b20000080400039
:108b0000c5f8070095fb07000080fa00000006008a
:108b10000800fa00889fbe008a9fbe008083200064
:108b20005001be004000be00848320005403be00fc
:108b30004402be00c0ea07000004be000205be00f9
:108b4000008320005001be004000be0004832000ce
:108b50005403be004402be00b7ea07000002be0094
:108b60000203be000800be000a01be00edef0700d0
:108b700085eb0700009fbe000297be000083200027
:108b80005001be004000be00848320005403be009c
:108b90004402be001deb0700ffed07000483200028
:108ba000009abe000292be0008c8bf00e14f50000c
:108bb00007003a00008320005001be004000be00c4
:108bc0004afb070004832000009abe000292be0008
:108bd000808320003e02be002e03be000498be002b
:108be0000690be004f05be004f04be000080fa0094
:108bf000000006000800fa0008c8bf00e14f50005e
:108c00000c003a00008320005001be004000be006e
:108c100042fb0700deed0700848320005403be0002
:108c20004402be0084ea0700009fbe000297be0017
:108c30000a003700008320005001be004000be0043
:108c4000d3ed0700848320005403be004402be001d
:108c500079ea0700009fbe000297be0008c8bf0067
:108c6000e14f50000d003a00008320005001be008b
:108c70004000be0029fb0700b5ed070084832000fb
:108c80005403be004402be006bea070004832000c8
:108c9000009abe000292be000b0037000083200045
:108ca0005001be004000be00a9ed070084832000f3
:108cb0005403be004402be005fea070004832000a4
:108cc000009abe000292be00808320003e02be00d9
:108cd0002e03be000498be000690be000080fa007d
:108ce000000006000600fa0060632e0035f8070059
:108cf00070642e0048f80700d8f90700000f7800cc
:108d00001e00e000fcff32001e00780020079800e3
:108d10002e009000e50f50001c0032002e00900045
:108d2000e50f500007003c002e009000e30f5000bc
:108d30000e0032002e009000e40f50000f003200b1
:108d4000220037002e009000eb0f50001700320079
:108d50002e009000ec0f5000180032002e00900002
:108d6000ea0f50000d003200180037008e80e80036
:108d70001004200080087800190037008e80e80079
:108d80002004200080087800150037008e80e8005d
:108d90003004200080087800110037008e80e80041
:108da00040042000800878000d0037008e80e80025
:108db0005004200080087800090037008e80e80009
:108dc000600420008008780005003700a0812000a2
:108dd000fcf70700908020000ff80700190037000b
:108de00090802000d0dd0700ef0f500015003e00fe
:108df0002bc8bf00e14f500007003a0070418000cf
:108e00000000e00002003a000040eb0009e8b70073
:108e10000000eb00704188008e80e8009080200008
:108e200096de07000040eb002be8b7000040eb00a7
:108e30002ce8b700a0812000e2f707009080200016
:108e4000f5f707000080fa00000006002400fa0091
:108e50000000eb0030079800000037003e00900053
:108e6000700f98007e089000e30f50002c00320035
:108e70007e089000e30f50000a003c007e0890003e
:108e8000e10f5000180032007e089000e10f500002
:108e90001c003c007e0890000000e0000b00320047
:108ea0004b0037007e089000e50f50003000320084
:108eb0007e089000e50f5000200035007e089000ed
:108ec000e60f50003700320041003700ec00470049
:108ed00080652e000a000900b0587800b100b1008a
:108ee000b000b1003a003700ec00470030662e00b9
:108ef0000a000900b0587800b100b100b000b1001c
:108f000033003700ec004700e0662e000e00090039
:108f1000b0587800f100b100f000b1002c0037002b
:108f2000ec004700d0672e000e000900b058780012
:108f3000f100b100f000b100250037006c004700df
:108f400000017800b076260001d222000089be0020
:108f500064014100e0032200c12626000089be0012
:108f6000640141000040eb00004978001800370020
:108f70006c00470000017800c026260001d22200c4
:108f80000089be0064014100e0032200b1762600a2
:108f90000089be00640141000040eb0000497800f8
:108fa0000b0037006c0047000001780020142400fb
:108fb000315524000089be006401410000e2240014
:108fc000000978000281e8000040eb0000497800c9
:108fd0006c0047007bf70700c0682e008ef7070083
:108fe0001ef90700500798005e0090000000e000a6
:108ff000fbff32000000eb00000888005e009000dc
:10900000e70f5000180132005e009000f70f50008b
:10901000150132000000eb00104b88000000eb004f
:10902000000888005e009000f60f500003003a0030
:109030003e0090000000e800300798003e009000dd
:10904000e50f5000020034000000eb0030079800ec
:109050005e009000ef0f500003003a003e009000c9
:109060000000e900300798003e0090000000e0009a
:1090700002003d0050002000300798005e00900084
:10908000f90f500075ff3a003e009000001798005d
:109090000e109000e30f50004b0032000e109000b5
:1090a000e30f50000a003c000e109000e10f50004a
:1090b000200032000e109000e10f50002c003c0008
:1090c0000e1090000000e0000b00320063ff37003c
:1090d0000e109000e50f5000600032000e1090005e
:1090e000e50f50004e0035000e109000e60f5000c6
:1090f0006900320059ff37003bfc07000083200065
:109100005001be004000be0064aa20006554220049
:1091100056272000a7f9230047e907000483200011
:10912000009abe000292be001afa070062fc070015
:10913000cd0037002cfc0700008320005001be004a
:109140004000be00c45e2f00a5d72b00e6f52a0024
:109150003704240038e9070004832000009abe0089
:109160000292be000bfa070053fc0700be00370056
:109170001dfc0700008320005001be004000be001f
:109180006022b80006002000070424005eee0700fd
:109190006022b800060020004701240026e90700ed
:1091a0006022b800060020002702240097e907008b
:1091b00004832000009abe000292be00f5f9070069
:1091c0003dfc0700a800370007fc070000832000d3
:1091d0005001be004000be006022b8000600200022
:1091e0002702240014e907006022b80006002000ce
:1091f0004701240085e907006022b800060020002e
:109200000704240047ee070004832000009abe00f4
:109210000292be00dff9070027fc0700920037002a
:10922000f1fb0700008320005001be004000be009b
:10923000c45e2e0065f6220016312a0017002400b5
:10924000fde8070004832000009abe000292be00e1
:10925000d0f9070018fc070083003700e2fb070085
:10926000008320005001be004000be0014e5250030
:1092700075ab2400867a2000d7fd2300eee80700b6
:1092800004832000009abe000292be00c1f90700cc
:1092900009fc0700740037000000eb00200798006d
:1092a000000037002e009000101798001e1090004c
:1092b000e20f5000220032001e109000e20f50001a
:1092c00007003c001e1090000000e0000e0032007d
:1092d0001e109000e10f50001200320033003700e2
:1092e0001e109000e40f5000230032001e1090006a
:1092f000e40f5000190035001e109000e50f5000db
:109300002400320029003700ec004700c0692e001d
:109310000a000900b0587800b100b100b000b100f7
:1093200022003700ec004700706a2e000a00090096
:10933000b0587800b100b100b000b1001b00370098
:10934000ec004700206b2e000a000900b05878009e
:10935000b100b100b000b10014003700ec004700cc
:10936000d06b2e000a000900b0587800b100b1009f
:10937000b000b1000d003700ec004700806c2e00fb
:109380000a000900b0587800b100b100b000b10087
:1093900006003700ec004700306d2e000a0009007f
:1093a000b0587800b100b100b000b1006c004700c7
:1093b00084f60700e06d2e0097f6070027f80700f7
:1093c000400798004e0090000000e000fbff3200d4
:1093d0000000eb00000888004e009000e70f5000ee
:1093e000210032004e009000f60f500003003a00ba
:1093f0002e0090000000e800200798002e0090004a
:10940000e50f5000020034000000eb002007980038
:109410004e009000ef0f500003003a002e00900025
:109420000000e900200798002e0090000000e000f6
:1094300002003d0050002000200798004e009000e0
:10944000f90f500097ff3a002e0090000000e00056
:109450000100320093ff370063fb07006000b80093
:10946000008fbe00ffff37000080fa0000000600fa
:109470000000fa00008420005001be004000be0041
:1094800084842000009abe000292be0080832000e7
:109490005001be004000be0004842000009abe00bf
:1094a0000292be00008320005001be004000be00ba
:1094b00084832000009abe000292be006cfb07006d
:1094c0000080fa00000006000000fa00008420007e
:1094d0005001be004000be0084832000009abe0000
:1094e0000292be00808420005001be004000be00f9
:1094f00004842000009abe000292be000080fa00a0
:10950000000006001000fa00889fbe008a9fbe007f
:10951000400798000040800050079800de0090004f
:10952000e18f5000110032005e009000e10f50000a
:1095300004003c00de0090000100e0000800320062
:10954000b20037005e009000e20f50000a003200c7
:10955000de009000e38f50006e003200ab00370059
:109560004e00900094f90700a80037004e009000cc
:1095700008fa0700a50037004e0090006007980029
:10958000ee009000e38f5000300032006e0090003b
:10959000e30f500007003c00ee009000e18f500008
:1095a0000e0032006e009000e20f500018003200f2
:1095b00096003700ee009000e58f50003300320037
:1095c0006e009000e50f50002b003500ee0090007b
:1095d000e68f5000320032008c0037002bc8bf00ed
:1095e000e14f500001003a00a1ff0700f06e2e008d
:1095f0009180200010000900b05878001001b100df
:109600000040eb002be8b7002bfb07007f00370082
:10961000f5fa0700008320003002be002003be00e0
:10962000808320005001be004000be002ce90700ee
:1096300004832000009abe000292be00a2ff070031
:10964000d4f807001cfb070070003700e6fa07009b
:10965000008320005001be004000be00aeed0700b8
:1096600004832000009abe000292be00c9f80700e1
:1096700011fb070065003700dbfa070024fd070037
:10968000c4f807000cfb070060003700d6fa07009b
:1096900058fd0700bff8070007fb07005b00370015
:1096a000d1fa0700808320005001be004000be00b8
:1096b000048320005403be004402be00dee707001e
:1096c0000004be000205be00808320005001be00e1
:1096d0004000be00048320005403be004402be00cc
:1096e00010ed07000002be000203be000800be002d
:1096f0000a01be0045e8070004832000009abe006e
:109700000292be0070ff0700a2f80700eafa070005
:109710003e0037004e00900070079800fe00900059
:10972000e38f50001c0032007e009000e30f5000d9
:1097300007003c00fe009000e18f50000e00320058
:109740007e009000e20f50000f0032002f00370023
:10975000fe009000e58f50001c0032007e0090005b
:10976000e50f50000e003500fe009000e68f50001f
:1097700025003200250037009bfa07002ffc070068
:10978000cdfa07002100370097fa070072fc0700a6
:10979000c9fa07001d003700acfd07001b003700a9
:1097a00091fa0700008320005001be004000be0077
:1097b0005ffa070004832000009abe000292be00f8
:1097c00074f80700bcfa07001000370086fa07009b
:1097d000008320005001be004000be00545525000b
:1097e000555525005655250057fd2300bce80700b8
:1097f00004832000009abe000292be0065f80700b4
:10980000adfa07000100370036fd07004f05be0026
:109810004f04be000080fa00000006000200fa00bb
:10982000000f7800908020003fdb0700ef0f500012
:1098300019003e002cc8bf000004e00016003a00ea
:109840002bc8bf00e14f500008003a007041800073
:109850000000e00001003a0005ff07000040eb00b7
:1098600009e8b7000000eb00704188009e00780016
:109870009080200001dc07000040eb002be8b700df
:109880000040eb002ce8b700a08120004df5070058
:109890009080200060f507000080fa0000000600bc
:1098a0000a00fa000040eb0009e8b7000040eb00b6
:1098b0001ae8b7000040eb0003e8b7000040eb00f7
:1098c00004e8b7000040eb0005e8b7000040eb00fb
:1098d00002e8b7000000eb000040880010c0b300b1
:1098e0002be8b70050fa070061fa0700a0812000ba
:1098f00034f507009080200047f50700000037008e
:10990000d6f60700400798004e0090000000e000e7
:10991000fbff32000000eb00000888004e009000c2
:10992000f70f500003003a006009200095f407008b
:109930007e0137000000eb00104b88000000eb00b8
:10994000000888004e009000f10f500005003a001a
:109950002cc8bf000004e00002003a0000702e0096
:10996000aeff07004e009000f20f500005003a00d5
:109970002cc8bf000004e00002003a0020702e0056
:10998000a6ff07004e009000f30f500005003a00bc
:109990002cc8bf000004e00002003a0040702e0016
:1099a0009eff07004e009000ea0f500008003a00aa
:1099b0002cc8bf000004e00003003a0060702e00d5
:1099c00096ff07000200370040002000cdfe070090
:1099d0004e009000eb0f500008003a002cc8bf006a
:1099e0000004e00003003a0080702e008bff0700a7
:1099f0000200370050002000c2fe07004e00900019
:109a0000ec0f500008003a002cc8bf000004e00032
:109a100003003a00a0702e0080ff0700020037000c
:109a200060002000b7fe07004e009000e30f5000da
:109a300008003a002cc8bf000004e00003003a0010
:109a4000c0702e0075ff07000200370010002000d4
:109a5000acfe07004e009000e40f500008003a00f2
:109a60002cc8bf000004e00003003a00e0702e00a4
:109a70006aff07000200370020002000a1fe070057
:109a80004e009000e50f500008003a002cc8bf00bf
:109a90000004e00003003a0000712e005fff0700a1
:109aa000020037003000200096fe07004e009000b4
:109ab000f00f500005003a002cc8bf000004e00081
:109ac00002003a0020712e0054ff07004e00900063
:109ad000e90f500022003a009080200092da07003f
:109ae000ef0f50001e003e0003c8bf000004e0005e
:109af0001b003a0002c8bf000004e00018003a0052
:109b00002bc8bf00e14f50000a003a0090802000af
:109b100001c3b300014878000000e800e1c2b300cf
:109b2000014878000000e8008040eb000148780020
:109b30000300370041712e00908020004fdb0700aa
:109b400010c0b30003e8b7000040eb002be8b700fb
:109b5000a08120009bf4070090802000aef4070055
:109b60004e009000f90f500009003a002cc8bf00c9
:109b70000004e00006003a009bf907003cfe0700e5
:109b8000d6f90700100020007041880081f7070017
:109b90004e009000f60f500011003a002cc8bf0094
:109ba0000004e0000e003a008ff90700cbf907002f
:109bb000008320005001be004000be0084832000ce
:109bc0005403be004402be00d6eb0700048320000d
:109bd000009abe000292be003bfe07006df7070030
:109be0004e009000ef0f500011003a002cc8bf004b
:109bf0000004e0000e003a007bf90700b7f9070007
:109c0000808320005001be004000be00048320007d
:109c10005403be004402be00bbeb070004832000d7
:109c2000009abe000292be0027fe070059f7070007
:109c30004e009000e80f500011003a002cc8bf0001
:109c40000004e0000e003a0067f90700a3f90700de
:109c5000008320005001be004000be00848320002d
:109c60005403be004402be0073e6070004832000d4
:109c7000009abe000292be0013fe070045f70700df
:109c80004e009000e10f500011003a002cc8bf00b8
:109c90000004e0000e003a0053f907008ff90700b6
:109ca000808320005001be004000be0004832000dd
:109cb0005403be004402be00d4e607000483200023
:109cc000009abe000292be00fffd070031f70700b8
:109cd0004e009000e70f500027003a000040eb00d4
:109ce00006e8b7000040eb0007e8b7002cc8bf004b
:109cf000e14f500007003a000040eb002ce8b700ad
:109d0000a08120002ff407009080200042f407007b
:109d1000190037002bc8bf000004e00008003a001b
:109d20000040eb0009e8b700a081200025f40700ff
:109d30009080200038f4070068f907000e00370013
:109d4000808320005001be004000be00048320003c
:109d5000009abe000292be00dbfd07008484200052
:109d60006000b8006011b800009abe000292be0008
:109d700008f7070059f907004e009000f50f500052
:109d800001003a0038fb07004e009000f40f50002d
:109d90001c003a002cc8bf000004e00019003a0083
:109da00002c8bf000004e00016003a0010c0b30073
:109db00002e8b7002bc8bf00e14f50000a003a008c
:109dc0009080200011c3b300014878000000e80033
:109dd00051c6b300014878000000e8008040eb0065
:109de000014878000300370061712e009080200048
:109df000a2da07000040eb002be8b70090802000bb
:109e000005f407004e009000e60f500015003a00e0
:109e10002cc8bf000004e00012003a00f2f807006e
:109e2000008320003002be002003be00049fbe005d
:109e30000697be00808320005001be004000be0097
:109e400004832000009abe000292be00808320009e
:109e50003e02be002e03be000498be000690be0067
:109e6000ccf607004e009000ed0f500021003a00a4
:109e70002cc8bf000004e0001e003a00daf807001a
:109e8000008320003002be002003be00049fbe00fd
:109e90000697be00808320005001be004000be0037
:109ea00004832000009abe000292be0000842000bd
:109eb0005001be004000be0084832000009abe0016
:109ec0000292be00808420005001be004000be000f
:109ed00004842000009abe000292be00808420000c
:109ee0003e02be002e03be000498be000690be00d7
:109ef000a8f607004e009000f80f500006003a0048
:109f00002cc8bf000004e00003003a00b6f80700c8
:109f100001f907009ff607004e009000e20f500085
:109f200077fe3a00bbf9070075fe37000080fa00a3
:109f3000000006001000fa00889fbe008a9fbe0045
:109f400080458000e10f50000f003a0000832000a0
:109f50005001be004000be00848320005403be00b8
:109f60004402be00efea070004832000009abe000e
:109f70000292be00848320006000b8006011b80027
:109f8000009abe000292be0080458000e20f5000a1
:109f90000f003a00808320005001be004000be0048
:109fa000048320005403be004402be00d6ea07002a
:109fb00004832000009abe000292be008483200029
:109fc0006000b8006011b800009abe000292be00a6
:109fd00080458000e30f50000f003a00008320000e
:109fe0005001be004000be00848320005403be0028
:109ff0004402be0090e5070004832000009abe00e2
:10a000000292be00848320006000b8006011b80096
:10a01000009abe000292be0080458000e40f50000e
:10a020000f003a00808320005001be004000be00b7
:10a03000048320005403be004402be00f3e5070081
:10a0400004832000009abe000292be008483200098
:10a050006000b8006011b800009abe000292be0015
:10a0600080458000ed0f50001d003a0080832000e5
:10a070005001be004000be00048320005403be0017
:10a080004402be006ce507000004be000205be00ed
:10a09000808320005001be004000be0004832000e9
:10a0a0005403be004402be009eea07000002be0048
:10a0b0000203be000800be000a01be00d3e507008f
:10a0c00004832000009abe000292be008483200018
:10a0d0006000b8006011b800009abe000292be0095
:10a0e00080458000eb0f50001b003a0000832000e9
:10a0f0005001be004000be000df807000004be0085
:10a100000205be00008320005001be004000be00da
:10a11000848320005403be004402be007aea070094
:10a1200003f807000002be000203be000800be00e4
:10a130000a01be00b5e5070004832000009abe00b6
:10a140000292be00848320006000b8006011b80055
:10a15000009abe000292be0080458000ec0f5000c5
:10a160002a003a00008320005001be004000be00db
:10a17000eff7070040079800510798006207980022
:10a1800073079800808320005001be004000be008d
:10a19000e7f707000004be000205be0000832000b0
:10a1a0005001be004000be00848320005403be0066
:10a1b0004402be0054ea0700ddf707000002be00bb
:10a1c0000203be000800be000a01be001ae5070037
:10a1d0000002be000203be004e009000de009000b0
:10a1e0006e019000fe01900088e5070004832000c6
:10a1f000009abe000292be00848320006000b80076
:10a200006011b800009abe000292be008045800036
:10a21000ee0f50000f003a00008320003002be0015
:10a220002003be00808320005001be004000be001d
:10a230002be6070004832000009abe000292be00b5
:10a24000848320006000b8006011b800009abe004e
:10a250000292be0080458000ef0f500001003a00de
:10a260002bfa070080458000f00f500001003a00f3
:10a2700060fa07004f05be004f04be000080fa00e0
:10a28000000006000000fa0090458000e10f500039
:10a290000a003a00008420005001be004000be00c9
:10a2a000848320005403be004402be001dea070060
:10a2b00084832000009abe000292be009045800078
:10a2c000e20f50000a003a00008420005001be0056
:10a2d0004000be00848320005403be004402be0040
:10a2e00009ea070084832000009abe000292be00a3
:10a2f00090458000e30f50000a003a0000842000df
:10a300005001be004000be00848320005403be0004
:10a310004402be00c8e4070084832000009abe0007
:10a320000292be0090458000e40f50000a003a00ff
:10a33000008420005001be004000be008483200045
:10a340005403be004402be0030e5070084832000b1
:10a35000009abe000292be000000eb00904588000b
:10a36000048420006000b8006011b800009abe00ac
:10a370000292be000080fa00000006000800fa0009
:10a38000000f780000408000100798009e009000a9
:10a39000e18f5000110032001e009000e10f5000cc
:10a3a00004003c009e0090000100e0000800320024
:10a3b000bc0037001e009000e20f50000a0032007f
:10a3c0009e009000e38f500078003200b500370007
:10a3d0001e007800f8f50700b20037001e00780074
:10a3e0006cf60700af0037001e00780020079800c9
:10a3f000ae009000e38f50002e0032002e0090003f
:10a40000e30f500007003c00ae009000e18f5000c9
:10a410000e0032002e009000e20f500014003200b7
:10a42000a0003700ae009000e58f50003d003200e4
:10a430002e009000e50f500029003500ae0090007e
:10a44000e68f50004800320096003700f06e2e0074
:10a450009180200010000900b05878001001b10070
:10a460000040eb002be8b70093f707008d003700a2
:10a470005df70700008320005001be004000be00d1
:10a4800084832000009abe000292be000483200054
:10a490006000b8006011b800009abe000292be00d1
:10a4a000e0002000804588003af5070082f70700a9
:10a4b0007c0037004cf70700008320005001be00ed
:10a4c0004000be0014ea070004832000009abe008a
:10a4d0000292be002ff5070077f7070071003700e2
:10a4e00041f70700008320005001be004000be007d
:10a4f00084832000009abe000292be0004832000e4
:10a500006000b8006011b800009abe000292be0060
:10a51000f0002000804588001ef5070066f7070060
:10a520006000370030f70700008320005001be00b4
:10a530004000be0084832000009abe000292be004c
:10a54000048320006000b8006011b800009abe00cb
:10a550000292be0000012000804588000df5070032
:10a5600055f707004f0037001ff707000083200052
:10a570005001be004000be0084832000009abe004f
:10a580000292be00048320006000b8006011b80091
:10a59000009abe000292be00d000200080458800d4
:10a5a000fcf4070044f707003e0037001e00780067
:10a5b00030079800be009000e38f50001c0032006e
:10a5c0003e009000e30f500007003c00be009000ea
:10a5d000e18f50000e0032003e009000e20f50006c
:10a5e0000f0032002f003700be009000e58f5000b2
:10a5f0001c0032003e009000e50f50000e003500b8
:10a60000be009000e68f5000250032002500370084
:10a61000f5f6070089f8070027f707002100370043
:10a62000f1f60700ccf8070023f707001d003700fc
:10a6300006fa07001b003700ebf607000083200036
:10a640005001be004000be00b9f6070004832000a0
:10a65000009abe000292be00cef4070016f7070073
:10a6600010003700e0f60700008320005001be0014
:10a670004000be005455250055552500565525006f
:10a6800057fd230016e5070004832000009abe0052
:10a690000292be00bff4070007f707000100370071
:10a6a00090f907000080fa00000006000200fa009e
:10a6b000000f7800908020009bd70700ef0f50001c
:10a6c00016003e002cc8bf000004e00013003a0052
:10a6d0002bc8bf00e14f500007003a0070418000d6
:10a6e0000000e00002003a000040eb0009e8b7007b
:10a6f0000000eb00704188009e00780090802000f0
:10a700005ed807000040eb002be8b7000040eb00ec
:10a710002ce8b70090802000bff107000080fa000d
:10a72000000006000a00fa000040eb0009e8b7004c
:10a730000040eb001ae8b7000040eb0003e8b70068
:10a740000040eb0004e8b7000040eb0005e8b7006c
:10a750000040eb0002e8b7000040eb0006e8b7005d
:10a760000040eb0007e8b7000000eb000040880065
:10a7700010c0b3002be8b700abf60700bcf607002b
:10a78000a08120008ff1070090802000a2f1070037
:10a790000000370031f30700400798004e0090009a
:10a7a0000000e000fbff32004e009000f70f500069
:10a7b0009f0232000000eb00104b88004e0090001a
:10a7c000f10f500005003a002cc8bf000004e00063
:10a7d00002003a0000702e00b4ff07004e00900007
:10a7e000f20f500005003a002cc8bf000004e00042
:10a7f00002003a0020702e00acff07004e009000cf
:10a80000f30f500005003a002cc8bf000004e00020
:10a8100002003a0040702e00a4ff07004e00900096
:10a82000ea0f500008003a002cc8bf000004e00006
:10a8300003003a0060702e009cff07000200370002
:10a8400040002000cdfe07004e009000eb0f5000ae
:10a8500008003a002cc8bf000004e00003003a00e2
:10a8600080702e0091ff070002003700500020008a
:10a87000c2fe07004e009000ec0f500008003a00a6
:10a880002cc8bf000004e00003003a00a0702e00b6
:10a8900086ff07000200370060002000b7fe0700b7
:10a8a0004e009000e30f500008003a002cc8bf0093
:10a8b0000004e00003003a00c0702e007bff070098
:10a8c0000200370010002000acfe07004e00900090
:10a8d000e40f500008003a002cc8bf000004e0005c
:10a8e00003003a00e0702e0070ff070002003700fe
:10a8f00020002000a1fe07004e009000e50f500050
:10a9000008003a002cc8bf000004e00003003a0031
:10a9100000712e0065ff07000200370030002000a4
:10a9200096fe07004e009000f00f500005003a0020
:10a930002cc8bf000004e00002003a0020712e0085
:10a940005aff07004e009000e90f500022003a0025
:10a9500090802000f4d60700ef0f50001e003e004c
:10a9600003c8bf000004e0001b003a0002c8bf009b
:10a970000004e00018003a002bc8bf00e14f50006f
:10a980000a003a009080200001c3b300014878001b
:10a990000000e800e1c2b300014878000000e800d0
:10a9a0008040eb00014878000300370041712e0021
:10a9b00090802000b1d7070010c0b30003e8b700b3
:10a9c0000040eb002be8b700a0812000fdf007005d
:10a9d0009080200010f107004e009000f90f500009
:10a9e00019003a002cc8bf000004e00016003a002d
:10a9f000fdf5070039f607004efd07009045800081
:10aa00000000e0000d003200008320005001be0075
:10aa10004000be0084832000009abe000292be0067
:10aa200018fe0700808320005001be004000be00d9
:10aa300004832000009abe000292be000000eb00da
:10aa400080458800d3f307004e009000f60f5000b9
:10aa500018003a002cc8bf000004e00015003a00be
:10aa6000e1f507001df6070032fd07000083200016
:10aa70005001be004000be0084832000009abe004a
:10aa80000292be00904580000000e000010032000c
:10aa9000fcfd0700008320006022b8006033b8008e
:10aaa0000498be000690be0010002000804588007b
:10aab000b8f307004e009000ef0f500018003a0066
:10aac0002cc8bf000004e00015003a00c6f50700de
:10aad00002f6070017fd0700008320005001be00aa
:10aae0004000be0084832000009abe000292be0097
:10aaf000904580000000e00001003200e1fd070009
:10ab0000008320006022b8006033b8000498be00c3
:10ab10000690be0020002000804588009df30700bd
:10ab20004e009000e80f500023003a002cc8bf00f0
:10ab30000004e00020003a00abf50700e7f507004d
:10ab400080458000e10f5000030032008045800006
:10ab5000e20f500009003a008045800090458800cf
:10ab6000808320005001be004000be00048420000d
:10ab7000009abe000292be0001003700edfc070003
:10ab8000008320005001be004000be0084832000ee
:10ab9000009abe000292be00048320006000b8004c
:10aba0006011b800009abe000292be003000200082
:10abb0008045880077f307004e009000e10f5000b9
:10abc00023003a002cc8bf000004e00020003a0037
:10abd00085f50700c1f5070080458000e10f5000b2
:10abe0000300320080458000e20f500009003a0067
:10abf0008045800090458800808320005001be0081
:10ac00004000be0004842000009abe000292be00f4
:10ac100001003700c7fc0700008320005001be0080
:10ac20004000be0084832000009abe000292be0055
:10ac3000048320006000b8006011b800009abe00d4
:10ac40000292be00400020008045880051f30700ba
:10ac50004e009000e70f50001c003a000040eb004f
:10ac600006e8b7000040eb0007e8b7002cc8bf00bb
:10ac7000e14f500007003a000040eb002ce8b7001d
:10ac8000a08120004ff007009080200062f00700b4
:10ac90000e0037002bc8bf000004e00008003a0097
:10aca0000040eb0009e8b700a081200045f0070054
:10acb0009080200058f0070088f507000300370057
:10acc0006af0070033f3070084f507004e00900098
:10acd000f50f500001003a0063f707004e009000a6
:10ace000f40f50001c003a002cc8bf000004e00024
:10acf00019003a0002c8bf000004e00016003a0044
:10ad000010c0b30002e8b7002bc8bf00e14f5000ed
:10ad10000a003a009080200011c3b3000148780077
:10ad20000000e80051c6b300014878000000e800c8
:10ad30008040eb00014878000300370061712e006d
:10ad400090802000cdd607000040eb002be8b70034
:10ad50009080200030f007004e009000e60f500079
:10ad600015003a002cc8bf000004e00012003a00b1
:10ad70001df50700008320003002be002003be0046
:10ad8000049fbe000697be00808320005001be00d5
:10ad90004000be0004832000009abe000292be0064
:10ada000808320003e02be002e03be000498be0039
:10adb0000690be00f7f207004e009000ed0f500025
:10adc0007e003a002bc8bf000004e00006003a00f5
:10add00080712e00fbef0700803e200069ef070026
:10ade000a0812000f7ef07002cc8bf000004e0009e
:10adf00072003a002bc8bf00e14f50006f003a00cc
:10ae0000204680004046880000468000204688009a
:10ae1000e045800000468800c0458000e04588008d
:10ae2000a0458000c045880080458000a04588007e
:10ae3000304680005046880010468000304688002a
:10ae4000f045800010468800d0458000f04588001d
:10ae5000b0458000d045880090458000b04588000e
:10ae6000008920005001be004000be00048a20007e
:10ae7000009abe000292be00008820005001be0071
:10ae80004000be0004892000009abe000292be006d
:10ae9000008720005001be004000be000488200052
:10aea000009abe000292be00008620005001be0043
:10aeb0004000be0004872000009abe000292be003f
:10aec000008520005001be004000be000486200026
:10aed000009abe000292be00808320005001be0096
:10aee0004000be0004852000009abe000292be0011
:10aef000808920005001be004000be00848a2000ee
:10af0000009abe000292be00808820005001be0060
:10af10004000be0084892000009abe000292be005c
:10af2000808720005001be004000be0084882000c1
:10af3000009abe000292be00808620005001be0032
:10af40004000be0084872000009abe000292be002e
:10af5000808520005001be004000be008486200095
:10af6000009abe000292be00008420005001be0084
:10af70004000be0084852000009abe000292be0000
:10af8000848320006000b8006011b800009abe0001
:10af90000292be00048420006000b8006011b80076
:10afa000009abe000292be000000eb0090458800af
:10afb0000000eb008045880076f207004e0090000c
:10afc000ee0f50008c003a002cc8bf000004e000d7
:10afd00089003a0084f40700c0f40700d5fb07009d
:10afe000904580000000e0000d003200008320004a
:10aff0005001be004000be0084832000009abe00c5
:10b000000292be009ffc0700808320005001be001a
:10b010004000be0004832000009abe000292be00e1
:10b02000848320006000b8006011b800009abe0060
:10b030000292be000000eb0080458800a045800021
:10b0400080458800c0458000a0458800e04580001c
:10b05000c045880000468000e0458800204680000a
:10b060000046880040468000204688000000eb0033
:10b0700040468800b045800090458800d04580005b
:10b08000b0458800f0458000d0458800104680001b
:10b09000f045880030468000104688005046800009
:10b0a000304688000000eb005046880000852000f4
:10b0b0005001be004000be0084832000009abe0004
:10b0c0000292be00008620005001be004000be007b
:10b0d00004852000009abe000292be000087200076
:10b0e0005001be004000be0004862000009abe0051
:10b0f0000292be00008820005001be004000be0049
:10b1000004872000009abe000292be000089200041
:10b110005001be004000be0004882000009abe001e
:10b120000292be00008a20005001be004000be0016
:10b1300004892000009abe000292be00048a20000a
:10b140006000b8006011b800009abe000292be0014
:10b15000808520005001be004000be000484200015
:10b16000009abe000292be00808620005001be0000
:10b170004000be0084852000009abe000292be00fe
:10b18000808720005001be004000be008486200061
:10b19000009abe000292be00808820005001be00ce
:10b1a0004000be0084872000009abe000292be00cc
:10b1b000808920005001be004000be00848820002d
:10b1c000009abe000292be00808a20005001be009c
:10b1d0004000be0084892000009abe000292be009a
:10b1e000848a20006000b8006011b800009abe0098
:10b1f0000292be00e7f107004e009000f80f5000e9
:10b2000006003a002cc8bf000004e00003003a002a
:10b21000f5f3070040f40700def107004e00900050
:10b22000e20f50005bfd3a00faf4070059fd3700c9
:10b230000080fa00000006002a00fa00881f78004b
:10b240000000eb0030079800000037003e0090003f
:10b25000101798009e109000e48f50004f003200ad
:10b260001e119000e40f510011003c009e1190004f
:10b27000e18f5100280032001e109000e10f5000b5
:10b2800004003c009e1090000100e0001500320018
:10b29000710037001e119000e20f51002b003200a8
:10b2a0009e119000e38f5100350032006a00370094
:10b2b0001e109000e60f5000530032009e109000c8
:10b2c000e68f5000420035001e119000e70f51003c
:10b2d000540032009e119000e88f51005800320057
:10b2e0005d0037006c0047000001780030552600f3
:10b2f000410722000089be006401410040952600fc
:10b30000d15626000089be00640141000040eb00d8
:10b3100000497800500037006c00470000017800b9
:10b3200030552600410722000089be00640141001b
:10b3300040142600415726000089be0064014100e8
:10b340000040eb0000497800430037006c004700e4
:10b350000001780030142600c13626000089be00a6
:10b360006401410000d22400f14626000089be009d
:10b3700064014100500620000009780036003700c3
:10b38000ec00470090722e000c000900b0587800c5
:10b39000d100b100d000b1002f0037006c00470091
:10b3a0000001780030552600c16626000089be00e5
:10b3b0006401410000422500513627000089be008b
:10b3c0006401410040072000000978002200370096
:10b3d0006c00470000017800c034240041042200c2
:10b3e0000089be006401410040972600d156260026
:10b3f0000089be0064014100f0562700410720008b
:10b400000089be0014003700ec00470060732e0076
:10b4100010000900b05878001101b1001001b1000e
:10b420000d003700ec00470070742e000c0009007e
:10b43000b0587800d100b100d000b100060037004c
:10b440006c00470012242600f35627000288be0035
:10b4500041072000210098006c00470059ee0700ca
:10b4600040752e006cee0700fcef070050079800b7
:10b470005e0090000000e000fbff32000000eb00e7
:10b48000000888005e009000f70f50007102320043
:10b490000000eb00104b88000000eb000008880063
:10b4a0005e009000f60f500003003a003e0090004e
:10b4b0000000e800300798003e009000e80f5000c0
:10b4c000020034000000eb00300798005e0090009e
:10b4d000ef0f500003003a003e0090000000e9002a
:10b4e000300798003e0090000000e00002003d00a0
:10b4f00080002000300798005e009000f90f500097
:10b5000052ff3a003e00900020179800ae109000c5
:10b51000e48f50001e0132002e119000e40f510004
:10b5200011003c00ae119000e18f5100720032001a
:10b530002e109000e10f500004003c00ae1090006f
:10b540000100e0001500320040ff37002e1190008e
:10b55000e20f5100bd003200ae119000e38f5100a8
:10b56000dd00320039ff37002e109000e60f50004a
:10b57000d7013200ae109000e68f5000a8013500d0
:10b580002e119000e70f5100f8013200ae1190002b
:10b59000e88f5100180232002cff370050762e0041
:10b5a0001dee070060772e0006ee0700abef0700e8
:10b5b000400798004e0090000000e000fbff3200c2
:10b5c0004e009000e70f5000220232004e00900023
:10b5d00095ee070020079800a0ef070040079800ad
:10b5e0004e0090000000e000fbff32002e009000b3
:10b5f0004404dd004e0090008bee07000000440084
:10b60000200798007162200091407800c0cfb300fd
:10b6100000c060000004a00027e6b7002e009000e4
:10b620002031880040782e00e6ed07008bef070000
:10b63000400798004e0090000000e000fbff320041
:10b640004e00900078ee07002007980083ef070077
:10b65000400798004e0090000000e000fbff320021
:10b660002e0090004404dd004e0090006eee0700b6
:10b67000000044002007980040792e00d1ed07001b
:10b6800076ef0700400798004e0090000000e000b1
:10b69000fbff32002e0090004404dd004e009000bd
:10b6a00061ee070000004400200798006bef0700e0
:10b6b000400798004e0090000000e000fbff3200c1
:10b6c0002e0090004404dd004e00900056ee07006e
:10b6d000000044002007980071622000914078002b
:10b6e000c0cfb30000c0600027e6b7002e00900076
:10b6f00020318800d701370050762e00c6ed0700b4
:10b70000407a2e00afed070054ef07004007980085
:10b710004e0090000000e000fbff32004e00900061
:10b72000e70f5000cb0132004e0090003eee0700c4
:10b730002007980049ef0700400798004e0090004e
:10b740000000e000fbff32002e0090004404dd000a
:10b750004e00900034ee07000000440020079800df
:10b76000207b2e0097ed07003cef07004007980074
:10b770004e0090000000e000fbff32002e00900021
:10b780004404dd004e00900027ee07000000440056
:10b790002007980031ef0700400798004e00900006
:10b7a0000000e000fbff32002e0090004404dd00aa
:10b7b0004e0090001cee0700000044002007980097
:10b7c0007162200091407800c0cfb30000c06000db
:10b7d0000014a00027e6b7002e009000203188005a
:10b7e000e07b2e0077ed07001cef07004007980074
:10b7f0004e0090000000e000fbff32004e00900081
:10b8000009ee07002007980014ef07004007980092
:10b810004e0090000000e000fbff32002e00900080
:10b820004404dd004e009000ffed070000004400de
:10b830002007980027c6bf003040b30027e6b700b6
:10b840002e0090002031880082013700b07c2e004d
:10b8500071ed070000003700304b80000000e00071
:10b8600003003200907d2e0056ed070002003700e5
:10b87000907e2e0053ed0700f8ee07004007980079
:10b880004e0090000000e000fbff32004e009000f0
:10b89000f90f50006f0132004e009000f60f50007b
:10b8a000030032004e009000ef0f5000eaff3a0014
:10b8b000304b80008000eb00011798000000e00092
:10b8c00002003a0012002000021798008e1190002a
:10b8d000334b8800e0ff3700907f2e0039ed0700e2
:10b8e00080802e004ced0700dcee0700400798003a
:10b8f0004e0090000000e000fbff32004e00900080
:10b90000f90f500053013a0080812e002ded070001
:10b910000000eb00000f78000000eb00100798001b
:10b920000000eb0000088800ccee0700e70f500095
:10b93000480132001e0090008040eb0062ee0700dc
:10b940001e0fe800300620009e0f10000c0034008f
:10b95000ec0047001e009000801f780070822e00cf
:10b96000801f780001007800b3d30700e4875700f8
:10b970006c00470028ed07000000eb00000f780086
:10b980001e0090000000e80010079800e4ff370058
:10b99000a1cab300a0ff2f004bee0700a0ff2f00ad
:10b9a00061ee07000080fb00100798008040eb006c
:10b9b000a0ff2f0044ee0700a0ff2f005aee070063
:10b9c0000080fb00000f78009e009000a00a20007d
:10b9d000808f500002003a001e00e0000a00320092
:10b9e00040832e00f7ec070030842e000aed07009c
:10b9f0009aee0700400798004e0090000000e0001b
:10ba0000fbff320013013700f0842e00edec07003d
:10ba100030842e0000ed070090ee070040079800ec
:10ba20004e0090000000e000fbff3200d0852e00a9
:10ba3000e4ec0700b0862e00f7ec070000003700aa
:10ba400086ee0700400798004e0090000000e000de
:10ba5000fbff32004e0090006101b8000080eb0057
:10ba60008080eb000201400083814800321798007b
:10ba70004317980080012000010020003e11900033
:10ba8000ce119000800f5100818f5900ecff3e00d5
:10ba90003e109000ce109000006001004200370080
:10baa0004d003700280037002a0037002c003700ef
:10bab0005800370045003700380037002e003700a7
:10bac000180037001a0037001c0037004b00370001
:10bad0004d0037002e0037002400370008003700e3
:10bae0000a0037000c0037003e00370031003700f5
:10baf00024003700d70037003d0037003000370002
:10bb000000702e00c4ec0700cdff370020702e001f
:10bb1000c1ec0700caff370040702e00beec0700e2
:10bb2000c7ff370060702e00bbec0700c4ff370072
:10bb300080702e00b8ec0700c1ff3700a0702e0007
:10bb4000b5ec0700beff3700c0702e00b2ec070056
:10bb5000bbff3700e0702e00afec0700b8ff3700e6
:10bb600000712e00acec0700b5ff370020712e00ed
:10bb7000a9ec0700b2ff370040712e00a6ec0700c9
:10bb8000afff370080872e00a3ec0700acff370023
:10bb9000a0872e00a0ec0700a9ff3700c0872e0069
:10bba0009dec0700a6ff3700e0872e009aec070007
:10bbb000a3ff370000882e0097ec0700a0ff370096
:10bbc00050882e0094ec07009dff3700b0882e00af
:10bbd00091ec07009aff370010892e008eec0700c9
:10bbe00097ff370050892e008bec070094ff370039
:10bbf00090892e0088ec070091ff3700108a2e00f4
:10bc000085ec07008eff3700708a2e0082ec07005b
:10bc10008bff3700908a2e007fec070088ff3700eb
:10bc2000d08a2e0067ec0700100880004700de0075
:10bc3000ec004700801f7800d08b2e00801f78001a
:10bc400001007800fcd20700e48757006c00470031
:10bc500071ec070001ee0700400798004e009000cd
:10bc60000000e000fbff32004e009000f60f500095
:10bc700008003a0011088000f01f2d00808f50004e
:10bc800004003e0010088000015020000100400028
:10bc9000100888004e009000ef0f500008003a0096
:10bca0001108800000502000808f500004003600f2
:10bcb0001008800001b02f0001004000100888002b
:10bcc0004e009000f90f500062003200d6ff37009e
:10bcd000908c2e003bec070026c6bf000080fb00c6
:10bce000ec004700801f7800808d2e00801f7800b8
:10bcf00001007800d0d20700e48757006c004700ad
:10bd000045ec0700d5ed0700400798004e00900075
:10bd10000000e000fbff32004e009000f60f5000e4
:10bd200003003a0026c6bf000040e80026e6b70040
:10bd30004e009000ef0f500003003a0026c6bf00ef
:10bd40000040e90026e6b7004e009000f90f5000d1
:10bd500001003200e0ff370061622000914078006e
:10bd6000f0822f0058ed07003a003700b07c2e001b
:10bd700029ec070000003700204b80000000e000a5
:10bd800003003200008e2e000eec07000200370088
:10bd9000008f2e000bec0700b0ed07004007980065
:10bda0004e0090000000e000fbff32004e009000cb
:10bdb000f90f5000270032004e009000f60f50009f
:10bdc000030032004e009000ef0f5000eaff3a00ef
:10bdd000204b80008000eb00710f98000000e00015
:10bde00002003a0012002000720f9800fe09900035
:10bdf000234b8800e0ff37006c01470000722500ec
:10be0000114627000089be0030862600010220006e
:10be100020019800310198006c00470001902e002d
:10be200096d20700ec00470040ceb300804878006f
:10be30006c004700e3eb070080902e00f6eb070054
:10be400086ed0700400798004e0090000000e000db
:10be5000fbff32004f0478000080fa00000006006b
:10be60000800fa00300798003e009000000f7800ac
:10be7000000f20001e0060004400de001007980044
:10be8000be009000010f78009e0078006f80600077
:10be9000200798001e0090006a00b900800078001a
:10bea0002e009000008040000080fa000000060094
:10beb0000800fa00000f78001e0078006101b90048
:10bec000220798003307980090002000010020000e
:10bed0002e019000be019000800f5100818f59000b
:10bee0002b003e002e009000be009000006001007c
:10bef000090037000b0037000d0037000f00370036
:10bf00001100370013003700150037001700370005
:10bf1000190037001b0037000103200011079800ab
:10bf20001d00370012032000120798001a00370086
:10bf30002303200013079800170037003003200068
:10bf400010079800140037004103200011079800e3
:10bf50001100370052032000120798000e0037002e
:10bf600063032000130798000b00370070032000c4
:10bf7000100798000800370081032000110798007f
:10bf800005003700920320001207980002003700d6
:10bf9000a3022000130798001e0090000080fa0002
:10bfa000000006000000fa000500fc005705200014
:10bfb000373b8800a80a2000383b880027a6a80045
:10bfc00000000000000000000080fa0000000600f1
:10bfd0000000fa0011e1a8002016800001102000e6
:10bfe000010070002016880040062000e5ea0700e6
:10bff0000080fa00000006000000fa0091168000a0
:10c0000000f02f000080600090168800211680004c
:10c01000b0ff2f00008060002016880021168000ed
:10c0200070ff2f00008060002016880011e1a90039
:10c0300021168000f0ef2f0000806000201688009d
:10c040000080fa00000006000000fa00000037003f
:10c0500006c2bf00614060000004e000fcff3a003f
:10c0600006c2bf00644060000004e000f8ff3a0030
:10c0700006c2bf00684060000004e000f4ff3a0020
:10c0800006c2bf00704060000004e000f0ff3a000c
:10c0900009c2bf000044b2000004e000ecff3a0017
:10c0a0000080fa00000006004e00fa00750047000c
:10c0b00091912e0033000900315878004003b100ff
:10c0c0004103b100e096200008e907002097200016
:10c0d00032e9070071c9bf00f24f5000030036007b
:10c0e0001000200010079800020037000000eb004d
:10c0f00010079800204b8000e10f500048003a00e4
:10c1000071c9bf000080fb006101b900d0fe2f00a3
:10c11000f1ff2f0002014000838148005227980060
:10c120006327980010012000010020005e2190008c
:10c13000ee219000800f5100818f590038003e00a1
:10c140005e209000ee20900000600100110037009a
:10c1500013003700150037001700370019003700ab
:10c160001b0037001d0037002d0037002c00370062
:10c170002b0037002a00370029003700280037003d
:10c18000190037001b0037001d0037001f00370063
:10c190002100370010c0b30071e9b700200037005c
:10c1a00020c0b30071e9b7001d00370030c0b300f4
:10c1b00071e9b7001a00370040c0b30071e9b70059
:10c1c0001700370050c0b30071e9b7001400370002
:10c1d00060c0b30071e9b7001100370070c0b30050
:10c1e00071e9b7000e00370080c0b30071e9b700f5
:10c1f0000b00370090c0b30071e9b70008003700aa
:10c2000000c1b30071e9b7000500370010c1b300e9
:10c2100071e9b7000200370020c1b30071e9b7002f
:10c2200071c9bf000080fb00000f7800e4004700e8
:10c2300000c2b30080487800e400470000c2b300a9
:10c2400090409800e400470000c2b300a04098006e
:10c250001e0078004480de0015ff07008040780053
:10c26000640047003140980064004700b0409000ef
:10c2700000c3b30080cf500003003a00e400470041
:10c2800000c2b300b040980071c9bf000080fb003d
:10c290006f00600006ff07008040780064004700e0
:10c2a00041409800e4004700a0c3b300d04098008c
:10c2b00070c9bf000080fb00000f78001e007800ee
:10c2c0004480de00fafe07008040780064004700ea
:10c2d0006140980070c9bf000080fb006f006000e3
:10c2e000f3fe07008040780064004700714098002a
:10c2f000e4004700a0c3b300804898006fc9bf00a6
:10c300000080fb00000f78001e0078004480de00f3
:10c31000e7fe07008040780064004700114898005d
:10c320006fc9bf000080fb006f006000e0fe0700e7
:10c33000804078006400470021489800204b80002e
:10c34000e10f50000d003a006400470011c6b30031
:10c35000314898001e0090000000e0000300320009
:10c36000e400470000c7b300b0489800e40047006d
:10c37000d0c6b300c048980006003700e40047006c
:10c3800000c2b300b0489800e400470000c2b30008
:10c39000c0489800e40047000040eb00d0489800f7
:10c3a0006400470087ea0700e400470000c2b300ca
:10c3b0008048780073c9bf000080fb00000f780040
:10c3c0001e0078004480de00b9fe0700804078003f
:10c3d00064004700114098006400470090409000be
:10c3e00000c3b30080cf500003003a00e4004700d0
:10c3f00000c2b3009040980073c9bf000080fb00ea
:10c40000000f78009e0078006f806000a8fe070093
:10c41000804078006400470021409800e400470015
:10c4200040c7b300b0409800e400470080c6b300a6
:10c43000c040980073c9bf00e14f50000a003200ad
:10c44000319720009140780010c2b30080cf500097
:10c4500005003200319720009140780010c3b300ee
:10c4600080cf500006003a00e400470030c7b30018
:10c47000b0409800e400470040c7b300c0409800b7
:10c4800073c9bf00e24f5000050032003197200011
:10c490009140780020c2b30080cf500006003a00df
:10c4a000e4004700e0c6b300b0409800e400470055
:10c4b00040c6b300c040980073c9bf00e34f5000ae
:10c4c00005003200319720009140780030c2b3005f
:10c4d00080cf500006003a00e400470020c7b300b8
:10c4e000b0409800e400470040c6b300c040980048
:10c4f000e400470000c2b300d040980074c9bf00f8
:10c500000080fb0056fe0700000f7800c2002000ec
:10c510009e0f1100020034000000eb00000f7800b5
:10c520001e007800f50047004200dd00e0c0780002
:10c5300064004700614098001e007800f500470045
:10c540004200dd000000e800e0c078006400470021
:10c55000714098001e007800f50047004200dd00a1
:10c560000080e800e0c078006400470001489800bf
:10c57000e400470000c2b30090489800e400470080
:10c5800020c3b300a0489800e400470000c3b300f4
:10c59000b048980075c9bf000080fb00000f78000c
:10c5a0001e0078004480de0041fe070080407800d5
:10c5b000640047004148980075c9bf000080fb0037
:10c5c0006f0060003afe070080407800640047007a
:10c5d00051489800e40047000040eb00e048980014
:10c5e000640047000cea07000080fa000000060023
:10c5f0000000fa00316c20009140780000ceb300ba
:10c6000000c060002041b300c3e6b70021168000df
:10c610000020200000807000201688000080fa00b2
:10c62000000006000000fa00316c20009140780004
:10c6300000ceb30000c06000c3e6b7002116800042
:10c64000f0df2f0000806000201688000080fa00d4
:10c65000000006003600f800809fbe00829fbe00ea
:10c66000849fbe00869fbe003400f80000c0b30067
:10c67000a00188001200fa0005e1a9005efe070093
:10c68000e8ff0700c902a800c922a8008460a90029
:10c69000c962a900c0e2a9006060a8008660a90084
:10c6a000ad80a800ada0a900adc0a9009660a8000b
:10c6b0000040fe009660a9008660a90044fe0700c5
:10c6c0000000eb0000088800a5e907007fe90700eb
:10c6d000c902a900c922a9009eea070095ea07003d
:10c6e000ccc8bf000004e0000c0032000194200020
:10c6f0000e00780084cf07000e007800b1e9070033
:10c700000e007800afe90700119520000e007800b8
:10c710007dcf07000e007800bfe907000000eb00a6
:10c720000008880005e1a800401f200015e9070067
:10c730000080fa003400f9004f03be004f02be0033
:10c740004f01be004f00be003600f9000040060059
:10c750000000fa0021e3a9000080eb0060198800c6
:10c760000000eb00400388000000eb00500388004d
:10c770006960a8006840a8006a60a8006860a80016
:10c7800021e907000080eb00001688000080eb0024
:10c79000401688000080eb0080168800d002a900b7
:10c7a000d022a900d042a900d062a900d082a9005d
:10c7b000d0a2a900d0c2a900d0e2a900c042a9001d
:10c7c000c062a900c8c2a900c8e2a900d102a9009c
:10c7d000c902a900c922a900c102a900c122a90059
:10c7e0000000eb00101688000000eb0050168800d7
:10c7f0000481a80004a1a8000421a800510a200077
:10c8000091407800f0c8b30000c0600001c4b300dc
:10c8100001407000a5e0b70000e02100100888008a
:10c820000000eb000008880005e1a8009460a80063
:10c830001061a90011e1a8001081a90010a1a900b0
:10c8400010002000600888000000eb00300888001d
:10c8500010002000000c88008401a9008421a80099
:10c860008441a8008461a900216c200091407800d7
:10c8700000ceb30000c060002041b300c2e6b700a4
:10c880002200200061042000700520002374200095
:10c89000814978008049780082497800c1fd07000d
:10c8a00027e6a80010c0b30072e9b70010c0b300bb
:10c8b00073e9b70010c0b30074e9b70010c0b3004b
:10c8c00075e9b70010c0b30071e9b70010c0b3003c
:10c8d00070e9b70010c0b3006fe9b7004107a900c5
:10c8e000616c20009140780000ceb30000c0600071
:10c8f0003040b300c6e6b700416a2000914078009e
:10c9000000ceb30000c060005040b300a4e6b70002
:10c9100021e2a8002342a8002062a900c000200054
:10c920004011880020c2a90007e2a90010002000e1
:10c93000204b88000000eb00304b88000000eb002b
:10c94000404b88000000eb00504b88000040eb009b
:10c9500008e8b7000080fa00000006000400fa00b2
:10c960007bff0700fee80700d8e80700a6e80700fd
:10c97000a1168000f0ef2f0000806000a016880054
:10c98000f4e90700ebe90700f0822f0066ea0700f0
:10c9900026e6b70023ff070034e907000000370050
:10c9a00010002000104b8800bffd07000040eb0086
:10c9b000cce8b7000000eb00000f7800060037005d
:10c9c000a6ea0700204798002e4090000004e000ef
:10c9d00004003a001e0fe800100320009e0f100014
:10c9e000f7ff34002e409000f84f500011003a003d
:10c9f000fffe07000000eb00000f78000600370084
:10ca000096ea0700204798002e409000f84f50000b
:10ca1000040032001e0fe80070bb20009e0f1000c3
:10ca2000f7ff34002e409000f84f50000100320014
:10ca3000fcfe07002e409000f74f5000daff3a004e
:10ca400010c0b300cce8b700304b80000000e0001d
:10ca50000200320092f307000100370031f70700af
:10ca6000104b80000000e000cdff320020c0b3007a
:0cca7000cce8b700f0f90700c9ff370060
:020000040000fa
:020000040001f9
:0457f8001f7f00000f
:020000040000fa
:020000040001f9
:0457fc00703f0000fa
:020000040000fa
:10000800046b0000046b0000046b0000046b00002c
:10001800046b0000046b0000046b0000046b00001c
:10002800046b0000046b0000046b00002a630000ee
:10003800046b0000046b0000046b0000046b0000fc
:10004800046b0000046b0000046b0000046b0000ec
:10005800046b0000046b0000046b0000046b0000dc
:10006800046b0000046b0000046b0000046b0000cc
:10007800046b0000046b0000046b0000046b0000bc
:10008800046b0000046b0000046b0000046b0000ac
:10009800046b0000046b0000046b0000046b00009c
:1000a800046b0000046b0000046b0000046b00008c
:1000b800046b0000046b0000046b0000046b00007c
:1000c800046b0000046b0000046b0000046b00006c
:1000d800046b0000046b0000046b0000046b00005c
:1000e800046b0000046b0000046b0000046b00004c
:1000f800046b0000046b0000046b0000046b00003c
:10010800046b0000046b0000046b0000046b00002b
:10011800046b0000046b0000046b0000046b00001b
:10012800046b0000046b0000046b0000046b00000b
:10013800046b0000046b0000046b0000046b0000fb
:10014800046b0000046b0000046b0000046b0000eb
:10015800046b0000046b0000046b0000046b0000db
:10016800046b0000046b0000046b0000046b0000cb
:10017800046b0000046b0000046b0000046b0000bb
:10018800046b0000046b0000046b0000046b0000ab
:10019800046b0000046b0000046b0000046b00009b
:1001a800046b0000046b0000046b0000046b00008b
:1001b800046b0000046b0000046b0000046b00007b
:1001c800046b0000046b0000046b0000046b00006b
:1001d800046b0000046b0000046b0000046b00005b
:1001e800046b0000046b0000046b0000046b00004b
:0801f800046b0000046b000021
:020000040000fa
:10020800046b0000046b0000046b0000046b00002a
:10021800046b0000046b0000046b0000046b00001a
:10022800046b0000046b0000046b00002a630000ec
:10023800046b0000046b0000046b0000046b0000fa
:10024800046b0000046b0000046b0000046b0000ea
:10025800046b0000046b0000046b0000046b0000da
:10026800046b0000046b0000046b0000046b0000ca
:10027800046b0000046b0000046b0000046b0000ba
:10028800046b0000046b0000046b0000046b0000aa
:10029800046b0000046b0000046b0000046b00009a
:1002a800046b0000046b0000046b0000046b00008a
:1002b800046b0000046b0000046b0000046b00007a
:1002c800046b0000046b0000046b0000046b00006a
:1002d800046b0000046b0000046b0000046b00005a
:1002e800046b0000046b0000046b0000046b00004a
:1002f800046b0000046b0000046b0000046b00003a
:10030800046b0000046b0000046b0000046b000029
:10031800046b0000046b0000046b0000046b000019
:10032800046b0000046b0000046b0000046b000009
:10033800046b0000046b0000046b0000046b0000f9
:10034800046b0000046b0000046b0000046b0000e9
:10035800046b0000046b0000046b0000046b0000d9
:10036800046b0000046b0000046b0000046b0000c9
:10037800046b0000046b0000046b0000046b0000b9
:10038800046b0000046b0000046b0000046b0000a9
:10039800046b0000046b0000046b0000046b000099
:1003a800046b0000046b0000046b0000046b000089
:1003b800046b0000046b0000046b0000046b000079
:1003c800046b0000046b0000046b0000046b000069
:1003d800046b0000046b0000046b0000046b000059
:1003e800046b0000046b0000046b0000046b000049
:0803f800046b0000046b00001f
:020000040000fa
:10ca7c00507200006f670000726100006d200000b2
:10ca8c00537400006f720000656400002e000000fb
:10ca9c0020410000524300002020000048590000b3
:10caac0050200000284400004547000029000000e9
:10cabc002041000052430000202000004859000093
:10cacc0050200000285200004144000029000000c2
:10cadc00204900006e76000065720000736500004e
:10caec0000200000487900007065000072620000b0
:10cafc006f6c000069630000002000002020000023
:10cb0c002020000020200000202000002020000019
:10cb1c00202000002020000020000000252e000016
:10cb2c0039670000002500002e3800006700000067
:10cb3c0052450000434100004c4c000020520000c4
:10cb4c0045470000203000002d390000203f000038
:10cb5c0000200000535400004f52000045200000fc
:10cb6c005245000047200000302d00003920000005
:10cb7c003f00000020200000564100004c550000f2
:10cb8c0045200000535400004f5200004544000063
:10cb9c002020000000200000564100004c550000f1
:10cbac004520000052450000434100004c4c000061
:10cbbc0045440000200000004b6500007973000024
:10cbcc00747200006f6b000065200000526500005d
:10cbdc0063000000507200006f670000726100007b
:10cbec006d23000028300000302d00003539000086
:10cbfc0029000000507200006f6700007261000095
:10cc0c006d20000025320000690000005265000014
:10cc1c00632000004b65000079730000204e00007b
:10cc2c006f7700002e2e00002e0000004b650000d8
:10cc3c0079730000747200006f6b000065200000b7
:10cc4c00506c00006179000000520000756e00000d
:10cc5c006e6900006e6700002e2e00002e00000092
:10cc6c0020460000313d000041200000463200000b
:10cc7c003d42000020460000333d000043200000f0
:10cc8c0000200000463400003d4400002046000017
:10cc9c00353d000045200000463600003d460000b2
:10ccac00200000006d6900006c730000202d000056
:10ccbc003e2000006d6d0000006d00006d20000036
:10cccc002d3e0000206d0000696c00007300000018
:10ccdc004465000067200000462000002d3e000047
:10ccec002044000065670000204300000044000061
:10ccfc006567000020430000202d00003e2000004e
:10cd0c00446500006720000046000000434f00000f
:10cd1c004e5600003a2000002b2f00002d20000062
:10cd2c0026200000454e0000540000004465000021
:10cd3c00632000002d3e00002048000065780000b4
:10cd4c000044000065630000202d00003e20000020
:10cd5c00426900006e000000486500007820000069
:10cd6c002d3e0000204400006563000000480000d8
:10cd7c0065780000202d00003e2000004269000074
:10cd8c006e000000426900006e2000002d3e000085
:10cd9c00204400006563000000420000696e000042
:10cdac00202d00003e2000004865000078000000a7
:10cdbc0042410000534500004e3a0000202b000079
:10cdcc002f2d000020260000204500004e540000ae
:10cddc00003300002e3100003431000035390000e2
:10cdec00323600003533000035380000393700008a
:10cdfc003900000031000000320000003300000058
:10ce0c003400000035000000360000003700000040
:10ce1c003800000039000000300000002e00000037
:10ce2c006500000045520000523a0000204e000000
:10ce3c006f2000004f7000006572000061740000ec
:10ce4c006f720000004300006c650000617200000e
:10ce5c002045000045500000524f00004d000000de
:10ce6c00436c00006f6300006b430000616c0000ba
:10ce7c006962000072610000746900006f6e00004e
:10ce8c0000310000322f00003234000068720000c4
:10ce9c0020540000696d000065000000534500003f
:10ceac0054550000503a0000202b00002f2d00009c
:10cebc0020260000204500004e54000000280000f1
:10cecc0050720000657300007320000032200000d7
:10cedc0044690000676900007473000029000000b9
:10ceec00456e00007465000072200000486f000061
:10cefc0075720000733a000020000000456e0000bf
:10cf0c0074650000722000004d6900006e75000011
:10cf1c0074650000733a000020000000456e0000ac
:10cf2c00746500007220000053650000636f000000
:10cf3c006e640000733a000020000000456e000093
:10cf4c0074650000722000004d6f00006e740000cc
:10cf5c00683a000020000000456e00007465000077
:10cf6c007220000044610000793a000020000000ab
:10cf7c00456e0000746500007220000059650000c9
:10cf8c00617200003a20000000200000202b0000fd
:10cf9c002f2d000020260000204500004e540000dc
:10cfac004552000000430000616c0000632000004b
:10cfbc004d6f000064650000203d00002052000011
:10cfcc00504e000000430000616c00006320000024
:10cfdc004d6f000064650000203d00002041000002
:10cfec004c470000004500007261000073650000b2
:10cffc002045000045500000524f00004d2000001d
:10d00c003f000000454e0000544500005220000037
:10d01c006f72000020430000616e00006365000029
:10d02c006c0000004572000061730000696e000026
:10d03c006720000045450000505200004f4d000095
:10d04c000025000035690000206f000066200000fc
:10d05c003635000035330000350000004545000032
:10d06c00505200004f4d0000206600006169000026
:10d07c006c65000064210000005000007265000027
:10d08c0073730000204500004e5400004552000010
:10d09c000045000045500000524f00004d2000009c
:10d0ac00706100007373000065640000004b0000a9
:10d0bc0065790000626f000061720000642000005e
:10d0cc005465000073740000004d00004f440000d4
:10d0dc0045200000746f0000206500007869000096
:10d0ec00740000002b0000002d0000005800000010
:10d0fc002f0000004d6500006e750000004500001b
:10d10c006e74000065720000004300006c65000046
:10d11c0061720000002b00002f2d00000045000064
:10d12c005850000000530000544f00002f520000d4
:10d13c00434c000000280000524f00004c4c0000f3
:10d14c0000290000005800002d590000002b0000a1
:10d15c002f2d000020410000646a000020540000c4
:10d16c00696d0000656f00007574000000250000fb
:10d17c003369000020530000656300006f6e0000ef
:10d18c0064730000002b00002f2d000020410000d4
:10d19c00646a0000757300007420000043410000b5
:10d1ac004c000000434100004c3d000025340000c1
:10d1bc0069000000546900006d650000204d0000fe
:10d1cc006f640000652000003d200000313200003b
:10d1dc0068000000546900006d650000204d0000df
:10d1ec006f640000652000003d2000003234000018
:10d1fc00680000005265000076200000312e00000f
:10d20c003300000028630000294400006176000010
:10d21c0069640000204c0000204a00006f6e000082
:10d22c00657300000020000020200000004a000070
:10d23c00616e00000046000065620000004d0000b9
:10d24c00617200000041000070720000004d00008f
:10d25c0061790000004a0000756e0000004a000071
:10d26c00756c000000410000756700000053000061
:10d27c0065700000004f000063740000004e000059
:10d28c006f760000004400006563000000000000a1
:020000040000fa
:10d29c0076090000880000000200000020312f00f9
:10d2ac0078202000785e3200202053005152540028
:10d2bc002000200053494e00202043004f532000f3
:10d2cc00205441004e202000002050004920200016
:10d2dc0020585e0059202000655e78002020000058
:10d2ec0020524500432050004c415900202043005f
:10d2fc004f4e5600200020004c4f4700203130008c
:10d30c005e782000204c4f00476520000020410033
:10d31c00524320002048590050202000202020009b
:10d32c002020000020523e0050202000503e520091
:10d33c00202020002f2f200020002000207821000a
:10d34c00203352004f4f5400202041002d46200026
:10d35c000000000000080000760100000000000042
:10d36c00300b00000200000000000000de0a00008c
:10d37c00200000000200000000000000000000007f
:10d38c00b0410000000000000000700043000000ed
:10d39c0000006500cdcd410000c84e00676dc10096
:10d3ac00ab430000fe0a0000200000000200000059
:10d3bc000a000000006400000000e8000300000008
:10d3cc001027000000a0860001004000420f000062
:10d3dc00809698000000e100f50500008e0a000020
:10d3ec002e000000020000000001020003040500f2
:10d3fc0006070800090a0b000c0d0e000f0a0b00a3
:10d40c000c0d0e000f30310032333400353637003e
:10d41c003839610062636400656641004243440030
:10d42c004546000000000000fe0900004800000016
:10d43c00020000000000000000000000244000007a
:10d44c000000000000005900400000000000000037
:10d45c0088c34000000000000084d7009741000002
:10d46c0080e0370079c3410043176e0005b5b50065
:10d47c00b8934600f5f93f00e9034f00384d3200f0
:10d48c001d30f900487782005a3cbf00737fdd00e5
:10d49c004f1575001e0b000012000000020000006a
:10d4ac000100020000040000080010000000000051
:10d4bc00202b2d0023300000680b0000080000001a
:10d4cc0002000000686a6c00747a4c0000000000d6
:10d4dc00460a0000480000000200000000000000a6
:10d4ec000000000024400000000000000000590073
:10d4fc00400000000000000088c340000000000055
:10d50c000084d7009741000080e0370079c34100c8
:10d51c0043176e0005b5b500b8934600f5f93f000a
:10d52c00e9034f00384d32001d30f9004877820076
:10d53c005a3cbf00737fdd004f157500360b0000a1
:10d54c0032000000020000004e414e00006e6100ef
:10d55c006e0049004e460000696e660000303100d6
:10d56c003233340035363700383961006263640079
:10d57c006566000030313200333435003637380000
:10d58c00394142004344450046000000bc0a0000fb
:10d59c00220000000200000030313200333435002c
:10d5ac00363738003961620063646500660030000c
:10d5bc0031323300343536003738390041424300bc
:10d5cc004445460000000000320b00000200000041
:10d5dc000200000000000000700b000002000000c0
:10d5ec000200000030000000340b000002000000bc
:0cd5fc0002000000000000000000000021
:020000040000fa
:04d608000000fe0020
:00000001FF
